:020000040800F2
:10000000586000209D010008454C0008AD3D0008E7
:10001000BD4A00080D0A00085556000800000000FF
:10002000000000000000000000000000E14E000899
:100030006D12000800000000714E0008154F000806
:10004000B7010008B7010008B7010008B7010008B0
:10005000B7010008B701000871120008B7010008D5
:10006000B7010008B701000879120008B7010008BD
:10007000E50F0008B7010008B7010008B701000844
:10008000B7010008B7010008B7010008B701000870
:10009000110A00081D0A0008B701000881120008B3
:1000A000B7010008B7010008B7010008B701000850
:1000B000B7010008B7010008B7010008B701000840
:1000C000B7010008B7010008B7010008B701000830
:1000D000B701000855550008B70100086155000830
:1000E000B7010008B7010008B7010008B701000810
:1000F000B7010008B7010008B7010008B701000800
:10010000B7010008B7010008B7010008B7010008EF
:10011000B7010008B7010008B7010008E54F000863
:10012000B7010008F10F0008FD0F000809100008D2
:10013000B7010008B7010008B7010008B7010008BF
:10014000290A0008350A0008B7010008B7010008AD
:100150001510000821100008B701000839560008E2
:10016000B7010008B7010008B7010008B70100088F
:10017000B7010008B7010008B7010008000000003F
:10018000B7010008B7010008DFF80CD000F056FAFC
:1001900000480047F1560008586000200648804794
:1001A00006480047FEE7FEE7FEE7FEE7FEE7FEE75C
:1001B000FEE7FEE7FEE7FEE7D14F000889010008F1
:1001C0002DE9F05F0546002092469B46884606468C
:1001D000814640241BE0284641464746224600F01F
:1001E0006DF953465A46C01A914110D3114618462C
:1001F000224600F054F92D1A67EB01084F462246BB
:100200000120002100F04BF917EB00094E41201EA0
:10021000A4F10104DFDC484631462A464346BDE8E6
:10022000F09F00000649074A0868504343F239022C
:10023000104408604008704701490860704700009A
:10024000000000206D4EC64140EA01039B0703D029
:1002500009E008C9121F08C0042AFAD203E011F805
:10026000013B00F8013B521EF9D27047D2B201E0C7
:1002700000F8012B491EFBD270470022F6E710B5AB
:1002800013460A4604461946FFF7F0FF204610BD04
:100290002DE9F04D81EA030404F0004B21F0004504
:1002A00014464FF0000A23F0004150EA050220D026
:1002B00054EA01021DD0C5F30A570246C5F31303E1
:1002C000C1F31300C1F30A5640F4801543F48013C0
:1002D000A7EB0608101BD64608F2FD3873EB0500A5
:1002E00002D308F1010801E092185B41B8F1000F58
:1002F00003DA00200146BDE8F08D00204FF48011A4
:10030000064684460EE0171B73EB050705D3121B48
:1003100063EB050306434CEA010C49084FEA300041
:1003200092185B4150EA0107EDD152EA030012D066
:1003300082EA040083EA0501084305D0101BAB41A3
:1003400006D20122002306E000224FF0004302E023
:100350006FF0010253101AEB06004CEB085110EB42
:100360000A0041EB0B01BDE8F04D00F0EEB830B5EE
:10037000041E71F1000404DB4FF00044404264EBC2
:100380000101141E73F1000405DB1C464FF000430D
:10039000524263EB0403801A994101D3012030BD1E
:1003A000002030BD30B5041E71F1000404DB4FF0B5
:1003B0000044404264EB0101141E73F1000405DBAC
:1003C0001C464FF00043524263EB0403101A8B416A
:1003D00001D3012030BD002030BD30B5041E71F1C5
:1003E000000404DB4FF00044404264EB0101141EA2
:1003F00073F1000405DB1C464FF00043524263EBEF
:100400000403801A994101D2012030BD002030BD83
:1004100030B4044696230800214604D0B62330BCED
:10042000002200F064B820460021F8E70EB540F243
:10043000334102910021CDE900110A460B4600F03C
:1004400093F803B000BDC1F30A5210B5C1F3130114
:1004500040F2FF3341F480119A4201DA002010BDCE
:1004600040F233439A42A2F2334203DC524200F09C
:1004700025F810BD904010BD00F0004230F0004063
:100480000AD0C10D01F56071C0F3160042EA0151B6
:10049000C208400711437047002001467047202AD8
:1004A00004DB203A00FA02F1002070479140C2F1CB
:1004B000200320FA03F3194390407047202A04DBFD
:1004C000203A21FA02F00021704721FA02F3D040CD
:1004D000C2F1200291400843194670470029A8BF85
:1004E0007047401C490008BF20F00100704710B45D
:1004F000B0FA80FC00FA0CF050EA010404BF10BC12
:10050000704749B1CCF1200421FA04F411FA0CF13E
:1005100018BF012121430843A3EB0C01CB1D4FEA77
:1005200000614FEA102042BF002010BC704700EB72
:10053000C35010440029A4BF10BC7047401C4900A0
:1005400008BF20F0010010BC704710B5141E73F1F5
:10055000000408DA401C41F1000192185B411A4383
:1005600001D120F0010010BD2DE9F04D92469B46CF
:1005700011B1B1FA81F202E0B0FA80F22032904675
:10058000FFF78DFF04460F4640EA0A0041EA0B01DF
:1005900053465A46084313D0114653EA010019D076
:1005A000C8F140025046FFF789FF05460E46504607
:1005B00059464246FFF773FF084305D0012004E087
:1005C00020463946BDE8F08D0020054346EAE07636
:1005D0002C4337430A986305E40AA0EB0800002285
:1005E000FD0A44EA47540A3002D500200146E9E7F3
:1005F000010510196941DDE9084500196941BDE8A7
:10060000F04DA2E7002801DBC0F10040002901DB2A
:10061000C1F10041814202D24FF0004004E04FF0AE
:10062000005001D14FF0C040EFF3008121F07F4135
:1006300041EA000181F3008870470000064C074D35
:1006400006E0E06840F0010394E8070098471034A2
:10065000AC42F6D3FFF79CFD708B0008908B00082E
:10066000B4EEE00AB1EE602AB0EE401AF1EE10FAF4
:10067000B4EEC02AC8BFB0EE601AF1EE10FAC8BFDF
:10068000B0EE421AB0EE410A704700002DE9F04189
:1006900040F240240746984615460E46C2F2000432
:1006A000207801281EBFFD2040B2BDE8F08175B35F
:1006B000A068642105F0BAF900281EBFFB2040B2F3
:1006C000BDE8F081E06818B91AE000BF0069B8B170
:1006D0000178B94204BF4168B142F7D18668A06889
:1006E00005F0CEF97EB1304629460022434605F09A
:1006F000D7F8002818BF4FF0FF3040B2BDE8F081B6
:10070000A06805F0BDF9FC2040B2BDE8F081FE20F4
:1007100040B2BDE8F08100002DE9F04140F24027F1
:10072000064614460D46C2F20007387801281EBF5F
:10073000FD2040B2BDE8F081B868642105F076F98B
:10074000002C08BF0A2400281EBFFB2040B2BDE8D1
:10075000F081F86810B908E0006930B10178B14261
:1007600004BF4168A942F7D12BE0142000F0EAF859
:100770008046B8F1000F1AD020461C21002205F057
:10078000CFF80028C8F8080018D088F80060C8F82A
:10079000045088F80C40F868C8F81000C7F80C80BE
:1007A000B86805F06DF9002040B2BDE8F081B86886
:1007B00005F066F9FE2040B2BDE8F081404600F049
:1007C000BFF8B86805F05CF9FF2040B2BDE8F081E1
:1007D0002DE9F0418AB0044640F24020C2F2000008
:1007E0000078012803D1012C03D9FF2094E0FD20DB
:1007F00092E001F0FE00022802D00BB9FE208BE04F
:10080000DDF840C0BCF1080F01D9FF2084E040F6BC
:10081000CC1540F6A4160020012CC2F20005C2F24D
:10082000000618BF0546002C18BF2E4696B10329B6
:10083000CDE90800CDE90600CDE90400CDE90200CC
:1008400069D8DFE801F002090C1100200DF1080E53
:1008500000210EE0FE205FE002A8002106E0022158
:1008600000200DF1080E04E002A8022100F1040EA0
:100870000420CEF8002004AA002B82E803104FF0D9
:1008800000008DF81C0018BFBCF1000F05D002A8B5
:10089000194662461830FFF7D7FC304600F05EFD7F
:1008A00038B102A901AB304601F1180200F0F0FCAA
:1008B00078B341F24C1104EBC410C2F2000101EB19
:1008C000C002D2F80004D2F80434013000F01F0056
:1008D000984201D1FF201FE004EBC41302F58068A9
:1008E00001EBC301D8F80030DDE906C4DDE9025EA2
:1008F000DDE904725E018D5101EB43114C61C1E9E8
:10090000032CC1E901E7DDE90823C1E90623C8F8A2
:100910000000002000E0FF2040B20AB0BDE8F081F6
:10092000002904BF6FF00100704780B582B00B79D9
:100930000A6800934B1D0021FFF74AFF02B080BDFB
:1009400006F032B805F050BD2DE9F04104F036FF55
:100950004FF47A78B8FBF0F507F080FA4EF21807FA
:1009600005FB00F6CEF200073C6807F077FA684313
:100970003968864200FB08F008BF214657F8042C6E
:1009800000F57A7001FB08F10132B1FBF2F1401A77
:100990000021BDE8F081000040F6B43240F66C3131
:1009A0000128C2F20002C2F2000118BF0022002892
:1009B00018BF1146084670470068016811F0100F13
:1009C00008BF704781B000210323009101680091A6
:1009D0004168009144F60001C4F2000101F54C4267
:1009E000904208BF0123884240F2686108BF00239B
:1009F000C2F2000103EBC30001EB80000099006A22
:100A0000002801B000D0004770470000FEE700005A
:100A100040F6A410C2F2000000F0B6BC40F6A410EC
:100A2000C2F2000000F0B0BC40F6CC10C2F20000F0
:100A300000F0AABC40F6CC10C2F2000000F0A4BC4A
:100A40002DE9F04381B02DED048B04468946904694
:100A5000FE20002C18BFB9F1000F00F04481D4E94A
:100A600000010025B8EB000065EB0101FFF7D0FCA9
:100A70009FEDA00A01EE100A81EE001A9FED9E0A7A
:100A800011EE100A84ED021AC4E9008500F0FF405F
:100A9000B0F1FF4F0BD0B5EEC01AF1EE10FA06DD43
:100AA0009FED960AB4EEC01AF1EE10FA02DA84ED68
:100AB000020A08E09FED920AB4EEC01AF1EE10FAB5
:100AC000C8BF84ED020A207C99F80070B84237D084
:100AD000042F10D104280ED04046FFF7ADFBFFF7DE
:100AE000A1FB022121EA4000013800EE100AB8EE15
:100AF000C00A84ED0F0A94F9110001281FDB9FED55
:100B0000818A0026002500BFC6EB061004EB80009A
:100B1000503004F099F904EB4616B0EE480A06F599
:100B2000BE7003F0C9F906F5FE70B0EE480A03F096
:100B3000C3F994F911000135EEB28642E4DB277463
:100B4000052F07D0012F0ED19FED6E0A0020C4E9BA
:100B5000050072E0D9F804009FED6A0A6061D9F8D7
:100B60000800A06169E094ED0C0A94EDA61A31EE3C
:100B7000408AB0EE480A07F051FCB0EE409AB0EE61
:100B8000480A07F017FD99ED011A99ED022A29EE9E
:100B9000013A29EE024A00EE423A00EE014A84EDA3
:100BA000053A84ED064A207C062848D89FED550A70
:100BB000DFE800F04343041122430400D4ED021A9D
:100BC00094ED0C0AD4EDA60A9FED4E1A04F5A07020
:100BD00004F03AF831E094ED0C0A9FED4E2AD4ED82
:100BE000021AD4EDA60A9FED471A04F5A07030EE64
:100BF000020A04F029F820E09FED3F0A94ED0F8AE5
:100C000001EE108AB8EE411A21EE000A07F0D2FC7C
:100C10009FED3D1A20EE010A07F0F9FB9FED3B1A0C
:100C20009FED3B2A30EE010AB4EEC20AF1EE10FA53
:100C3000C8BFB0EE420A28EE000A84ED070A94F914
:100C400011309FED350A04F1120004F1140104F192
:100C5000400203F035FF94F91100012842DB9FEDBB
:100C6000298A9FED2E9A0025002600BF04EB05106F
:100C700004EB451790EDAA0A07F5BE7003F098F84B
:100C8000207CB0EE401A411E052911D204EB8501EB
:100C9000D4ED021AC5EB0510F0EE410AB0EE481A89
:100CA00091ED100A04EB8000503003F0CDFF09E015
:100CB0000628B0EE480A02BF04EB850090ED100A4A
:100CC00080EE090A07F5FE7003F072F804EB850068
:100CD000013680ED9F0AF5B294F911008542C5DB1B
:100CE000002000E0002040B2BDEC048B01B0BDE864
:100CF000F08300BF00007A446F12833A6F12033A08
:100D0000CDCC4C3D00000000CDCC4C3E9A99193F13
:100D1000CDCC4C3FAB611C3F00C0DA4500A00C4677
:100D20002DE9F04381B02DED028B0446B0EE408AF0
:100D3000894684B30020C4F80C9004F1300C207470
:100D400092E80B008CE80B0004F5267307CA07C372
:100D500099F86C0068B104F1300004F5267500F0D4
:100D60002FF99FED4F0A95ED001A30EE410A85EDFF
:100D7000000A99F86010FC27062900F28A804FF0DB
:100D800001080420DFE801F0040F090409850C00C4
:100D90000420884607E0FE277BE00846884602E0FC
:100DA0004FF005080120002509F120070026607496
:100DB000C4E90055A56000BFC5EB05100021B0EEE9
:100DC000480A3A4604EB8000503003F0F3FFD9EDB7
:100DD000190A04EB4515B0EE480A05F5BE7003F09C
:100DE00017F8D9ED1A0A05F5FE70B0EE480A03F0BF
:100DF0000FF894F911000136F5B28542DCDB04F5F9
:100E0000A07009F140020021B0EE480A002703F06B
:100E1000D1FF04F11200414603F00CFFC4E905774D
:100E2000E76194F91100012833DB0022002100BFA3
:100E300004EB02120131C2E9A977C2E9AB77CAB269
:100E40008242F5DB01280BDB00210023002200BFDA
:100E500004EB83030132C3F87C12D3B29842F7DC6F
:100E6000012815DB04F1200500260027E068304446
:100E700003F00CF9E068304403F0E2F845F827008D
:100E80000137083694F911008742EFDB002700E0B4
:100E9000002778B2BDEC028B01B0BDE8F08300BF43
:100EA000DB0FC940B0B5044634B394F911100129E1
:100EB00022DB0020002500BF04EB8002106A20B175
:100EC00092ED9F0A03F050F9617C01354AB2E8B215
:100ED0009042F1DB012A0FDB0020002105E000BF7A
:100EE0000131C8B29042A8BFB0BD04EB8000006AD7
:100EF0000028F5D003F01CF8B0BD000070B5044622
:100F0000FE20002C18BF002937D0E06891ED030ABD
:100F100090F86C10B1EE401A002918BFB0EE410AEB
:100F200084EDA60A94F91110012928DB03F088F951
:100F3000206A002802BFFE2040B270BD00250026B6
:100F400004EB061100F1080601354CCE406901F5AD
:100F5000297C8CE84C00C1F8B002EEB294F9110083
:100F600086420CDAE06800EBC60003F069F904EB96
:100F70008600006A0028E3D1FE2040B270BD002048
:100F800040B270BDB5EEC01A30EE600AF1EE10FA54
:100F9000D8BF7047B6EE002A21EE022AB4EEC20A8C
:100FA000F1EE10FAC4BF30EE410A7047B1EE422AAA
:100FB000B4EEC20AF1EE10FAB8BF30EE010A704783
:100FC0009FED040A90ED001A30EE410A80ED000A10
:100FD000704700BFDB0FC94040F21800C2F20000AA
:100FE0007047000040F22040C2F2000000F0EABD6D
:100FF00040F21050C2F2000000F0E4BD40F2900058
:10100000C2F2000000F0DEBD40F2C030C2F20000CB
:1010100000F0D8BD40F2F000C2F2000000F0D2BDF6
:1010200040F2C050C2F2000000F0CCBD10B5002864
:1010300002BFFE2460B210BD0024342100F8244B0E
:10104000FFF71BF960B210BDB0B50446002C02BF1B
:10105000FE2040B2B0BD254655F8100F01466FF393
:10106000DF21A1F5B671B1F5A56F11D8C0F3CA2182
:10107000A1F5B671B1F5A56F0AD8A988800D40EA2F
:1010800081206FF3DF20A0F5B670B0F5A56F02D90F
:10109000FF2040B2B0BDC1F34A02FF2011F4405F0F
:1010A00000F0C28089B2B1F5804FC0F0BD80A2F5DA
:1010B000B671B1F5A56F00F2B78001202070FFF77F
:1010C00043FCC4E9020104F134002421FFF7D5F800
:1010D0002968A8889FED550A8A0DC1F3CA236FF3CA
:1010E000DF2101EE101A42EA802202EE103AB8EE39
:1010F000411AC0F34A016FF3DF22B8EE422A31EE03
:10110000003A9FED4B1A04EE102A05EE101A32EE4B
:10111000002A810BB8EE444A33EE033AB8EE455A42
:1011200032EE022A34EE004A35EE005A83EE013ADE
:1011300082EE012A84ED0B3A34EE043A35EE054A8C
:1011400084ED0C2A83EE012A84EE013A84ED092A0B
:1011500084ED0A3A84F83910C0F3013084F838007D
:10116000E08A6087208BA087608BE087207F002843
:1011700018BF012084F84000617F002918BF0121B9
:1011800084F84110E28B02F0010384F84230C2F38C
:10119000400384F84330C2F3800384F84430C2F340
:1011A000C00384F84530C2F3001384F84630C2F31C
:1011B000401384F84730C2F3801384F84830C2F3F8
:1011C000C01384F84930C2F3002384F84A30C2F3D4
:1011D000402384F84B30C2F3802384F84C30C2F3B0
:1011E000C02384F84D30C2F3003384F84E30C2F38C
:1011F000403384F84F30C2F38033D20B84F8503040
:1012000084F8512084F8520084F85310208C02EEA8
:10121000100A0020B8EE422A32EE000A30EE000A30
:1012200080EE010A84ED0D0A40B2B0BD000080C41A
:101230000000A54410B504460020FFF7ADFB04F103
:101240001001122202F0EEFC002818BF4FF0FF3010
:1012500010BD000080B502460120012104F038FCD9
:101260000138B0FA80F0400980BD000070470000EE
:10127000012000F04BBF0000102000F047BF00002D
:10128000202000F043BF000072B600BFFEE7000060
:1012900010B590F82040D0F800C0DCF808E0013C20
:1012A000E4B2012C0ED81EF0E05F11D0CEF3016045
:1012B000012484401C60D1E9023E7BB14C6843EAC2
:1012C000C4030DE000F1240301204FF4802123E04A
:1012D00000F1240301204FF400111DE00B685B05B1
:1012E0000CEB001043EA0E03C0F880310B69C0F824
:1012F000843100F5C073097D012901BF00F5C27179
:101300000C6844F480740C605168C0F88C1111684A
:10131000C0F88811002001211A681143196010BD1E
:10132000D0B1006846F20041C4F20001884208D002
:1013300046F60001C4F20001884218BF7047012040
:1013400000E0002040F240213422C2F2000110FBF4
:101350000210006C00B100477047000090F82010A8
:101360000139C9B2012984BF002070470068816833
:10137000C1F380618268C2F3C06280681144C0F327
:1013800000700844704700002DE9F04F81B004461A
:1013900020684669D0F804908768D0F80CB0D0F87F
:1013A00010A0D0F8188016F0010F03D100253007E7
:1013B0001CD423E0F90710D001218160B80709D4BB
:1013C000780700F19880380700F19B80204600F0F4
:1013D000D3FA02E0204600F0EDFA0025F80500F10E
:1013E0009580F80300F1B580300707D51BF0100099
:1013F0001FBF20681021C16045F40075700708D533
:101400001BF0080005D020680821C160204600F0CC
:101410001DFAB00707D52068C06810F0030F1CBF85
:10142000204600F031FA700607D51AF010001FBFF1
:1014300020681021016145F48065B00608D51AF0D6
:10144000080005D0206808210161204600F03AFA22
:10145000F00607D52068006910F0030F1CBF204676
:1014600000F04EFAB00308D519F0100005D020683E
:1014700010214160204600F061FAF00308D519F010
:10148000080005D0206808214160204600F028FBB4
:10149000300440F198805FEA497040F1918006F491
:1014A000807018F0020F08EA102040EA050001469B
:1014B00018BF41F0020116F4007F08BF014618F082
:1014C000040F0D4618BF45F0040516F4806F08BFE1
:1014D0000D4616F4006F18BF18F0700070D0103869
:1014E0000009052867D8DFE800F003585B5E6164F7
:1014F00045F008055FE04FF40065F8057FF571AF32
:1015000004E04FF48055F8057FF56BAF20684FF489
:1015100080718160B8050AD478050FD4380513D4DA
:10152000204600F065FAF8037FF55EAF11E0204633
:1015300000F07CFAF8037FF557AF0AE045F4005558
:10154000F8037FF551AF04E045F48045F8037FF5DB
:101550004BAF20684FF480318160B8030AD4780320
:101560000FD4380313D4204600F07EFA30073FF53D
:101570003DAF43E7204600F095FA30073FF536AF20
:101580003CE745F4004530073FF530AF36E745F41A
:10159000803530073FF52AAF30E745F010050AE007
:1015A00045F0200507E045F0400504E045F08005E2
:1015B00001E045F480752068816921F07001816146
:1015C000206804214160002D04BF01B0BDE8F08F08
:1015D000606A28436062204601B0BDE8F04FFFF723
:1015E0009FBE0000B0B50446002C04BF0120B0BD72
:1015F00094F8200010B9204600F076F820680168C1
:1016000041F00101016000F073FE05462068416869
:1016100011F0010F05D100F06BFE401B0B28F5D334
:1016200010E0016821F00201016000F061FE054652
:101630002068416811F0020F0DD000F059FE401BE8
:101640000B28F5D3606A052140F400306062012068
:1016500084F82010B0BD217E026822F080030129A9
:1016600008BF42F080030360617E026822F04003FD
:10167000012908BF42F040030360A17E026822F006
:101680002003012908BF42F020030360E17E0268C5
:1016900042F01003012908BF22F010030360217FEC
:1016A000026822F00803012908BF42F00803036022
:1016B000617F026822F00403012908BF42F004039D
:1016C0000360D4E901C2D4E9033561691A432A43AE
:1016D0001143ACF101021143C1610020012160629C
:1016E00084F82010B0BD000080B586B0002246F618
:1016F000000143F6400C0592CDE90322CDE9012219
:10170000C4F20001C4F2020C036840F20040C4F2CB
:1017100002008B424AD046F20041C4F200018B42E3
:1017200040F0928040F26061C2F200010A68531CEE
:10173000002A0B600DD100210091DCF8001041F06F
:101740000071CCF80010DCF8001001F0007100917D
:1017500000990021022300F5006000915CF8102C34
:1017600042F008024CF8102C5CF8102C02F0080231
:101770000092009A03220192CDE9023109210492DC
:10178000059101A900F0CEFC14200521002200F0F3
:101790002FFE142000F01CFE15200521002200F071
:1017A00027FE152000F014FE06B080BD0092DCF884
:1017B000001041F08061CCF80010DCF8001001F05E
:1017C00080610091009940F26061C2F200010A68F4
:1017D000531C002A0B600DD100210091DCF8001091
:1017E00041F00071CCF80010DCF8001001F000713D
:1017F00000910099002100915CF8102C42F0020247
:101800004CF8102C5CF8102C02F002020092009AA6
:10181000602201920222CDE90221032104910921D3
:10182000059101A900F07EFC40200521002200F076
:10183000DFFD402000F0CCFD41200521002200F01A
:10184000D7FD412000F0C4FD06B080BDD0B10068D6
:1018500046F20041C4F20001884208D046F6000179
:10186000C4F20001884218BF7047012000E0002048
:1018700040F240213422C2F2000110FB0210C06A83
:1018800000B1004770470000D0B1006846F2004147
:10189000C4F20001884208D046F60001C4F20001FB
:1018A000884218BF7047012000E0002040F240212C
:1018B0003422C2F2000110FB0210806A00B100471E
:1018C00070470000D0B1006846F20041C4F2000148
:1018D000884208D046F60001C4F20001884218BFD1
:1018E0007047012000E0002040F240213422C2F283
:1018F000000110FB0210406B00B100477047000070
:10190000D0B1006846F20041C4F20001884208D01C
:1019100046F60001C4F20001884218BF704701205A
:1019200000E0002040F240213422C2F2000110FB0E
:101930000210006B00B1004770470000D0B1006892
:1019400046F20041C4F20001884208D046F6000188
:10195000C4F20001884218BF7047012000E0002057
:1019600040F240213422C2F2000110FB0210806BD1
:1019700000B1004770470000D0B1006846F2004156
:10198000C4F20001884208D046F60001C4F200010A
:10199000884218BF7047012000E0002040F240213B
:1019A0003422C2F2000110FB0210C06900B10047EE
:1019B00070470000D0B1006846F20041C4F2000157
:1019C000884208D046F60001C4F20001884218BFE0
:1019D0007047012000E0002040F240213422C2F292
:1019E000000110FB0210006900B1004770470000C1
:1019F000D0B1006846F20041C4F20001884208D02C
:101A000046F60001C4F20001884218BF7047012069
:101A100000E0002040F240213422C2F2000110FB1D
:101A20000210006A00B1004770470000D0B10068A2
:101A300046F20041C4F20001884208D046F6000197
:101A4000C4F20001884218BF7047012000E0002066
:101A500040F240213422C2F2000110FB0210406922
:101A600000B1004770470000D0B1006846F2004165
:101A7000C4F20001884208D046F60001C4F2000119
:101A8000884218BF7047012000E0002040F240214A
:101A90003422C2F2000110FB0210406A00B100477C
:101AA00070470000D0B1006846F20041C4F2000166
:101AB000884208D046F60001C4F20001884218BFEF
:101AC0007047012000E0002040F240213422C2F2A1
:101AD000000110FB0210806900B100477047000050
:101AE000D0B1006846F20041C4F20001884208D03B
:101AF00046F60001C4F20001884218BF7047012079
:101B000000E0002040F240213422C2F2000110FB2C
:101B10000210C06B00B100477047000070B504466A
:101B2000A66D00F0E5FB054694F83500022825D1A6
:101B30002068016821F016010160416921F08001EF
:101B40004161216C09B9A16C19B1016821F008014A
:101B50000160016821F00101016000E02068006877
:101B600010F0010F0ED000F0C3FB401B0528F5D983
:101B700020206065032084F835000CE0802060653B
:101B8000012008E0E06D3F2101FA00F0B060012083
:101B900084F8350000200021C0B284F8341070BDF4
:101BA00090F8351002291FBF802141650120704740
:101BB000052180F835100068016821F001010160FD
:101BC00000207047F0B581B00446002048F2B513FC
:101BD0000821009040F21400C1F64E33C2F200001A
:101BE0000268D4E9166037688140A2FB03253942B8
:101BF0000DD02268136813F0040F08D0136823F087
:101C000004031360B160616D41F001016165012160
:101C10008140394209D02268526912F0800F1FBFFB
:101C2000B160616D41F0020161650421814039427A
:101C300009D02268126812F0020F1FBFB160616DF7
:101C400041F0040161651021814039421AD02068B9
:101C5000026812F0080F15D0B1600268016812F432
:101C6000802F06D1C9055EBF016821F0080101601F
:101C700001E0080301D4216C00E0A16C00291CBF25
:101C800020468847E16D202000FA01F23A4242D016
:101C90002068036813F0100F3DD0B26094F835301F
:101CA0000268052B1ED122F016020260426922F062
:101CB00080024261226C0AB9A26C1AB1026822F059
:101CC000080202603F208840B060012084F835009F
:101CD000002084F83400216D00293FD02046884739
:101CE00001B0F0BD016852030CD4C9050ED40168DF
:101CF00021F010010160012084F83500002084F8F3
:101D0000340003E0080301D4616C00E0E16B0029BA
:101D10001CBF20468847606D00B3606D10F0010F56
:101D200017D00521A80A84F8351021680A6822F026
:101D300001020A60009A01328242009203D80A68C6
:101D400012F0010FF6D1012084F83500002084F84C
:101D50003400E16C00291CBF2046884701B0F0BD6B
:101D60002DE9F041044600F0C3FA0546002C02BFFD
:101D70000126F0B2BDE8F081022084F83500002091
:101D800084F834002068016821F00101016000E05E
:101D90002068016811F0010F08D000F0A9FA401B7B
:101DA0000528F5D903252023032667E0016848F2BA
:101DB0003F02CFF2100201EA020CD4E90126D4E975
:101DC0000353D4E90578D4E9071E42EA0C023243F2
:101DD0002A431A433A4342EA08021143626A41EA3B
:101DE0000E01042A1DD1D4E90B3719433943016090
:101DF000014651F8143F23F007031343D4E90A2E98
:101E000042EA030CBEF1000F13D0B8F5005F3BD0DF
:101E1000B8F1000F4BD1022A4CD0012A40D042B970
:101E200048E00160014651F8143F23F0070343EAFC
:101E3000020C4AF6AB22C1F800C06FF00F01012579
:101E4000002651FA80F1CAF6AA22A1FB02235F29DB
:101E50004FF03F014FEA131248F61833C0F6000363
:101E60009A5C40F2FF3320EA03004FF0000388BF82
:101E700040F004009140C4E916028160F0B263654D
:101E800084F83550BDE8F081032AD2D801254023DB
:101E900006EB82070126DFE802F0020D0203EDE700
:101EA000AEF1C072B2FA82F252093AB9C1E7032A1E
:101EB00004D3BED1CEF30062002ABAD0012540235C
:101EC0000126DBE710B590F834C0BCF1010F48D013
:101ED0004FF0010CD0F858E080F834C090F835C0CD
:101EE000BCF1010F3AD14FF0020C80F835C04FF031
:101EF000000CC0F854C0D0F800C0DCF8004024F456
:101F00008024CCF80040CCF804308368402B0B468A
:101F100008BF1346CCF8083008BF0A46CCF80C209E
:101F20003F22C16D02FA01F1CEF80810DCF8001072
:101F300041F01601CCF80010006C00281EBFDCF840
:101F4000000040F00800CCF80000DCF8000040F091
:101F50000100CCF800000020C0B210BD002180F8C4
:101F600034100220C0B210BD10B5044614F0010FA9
:101F700036D1A0073ED4600746D420074ED4E006F1
:101F800056D4A0065ED4600666D420066ED4E00562
:101F900077D4A00500F18080600500F188802005DD
:101FA00000F19080E00400F19880A00400F1A0808E
:101FB000600407D540F22060C2F20000806B002868
:101FC00018BF8047200458BF10BD40F22060C2F205
:101FD0000000C06B002800F09780BDE8104000476B
:101FE00040F22060C2F200000068002818BF80475D
:101FF000A007C0D540F22060C2F20000406800286F
:1020000018BF80476007B8D540F22060C2F20000D8
:102010008068002818BF80472007B0D540F22060B4
:10202000C2F20000C068002818BF8047E006A8D5AB
:1020300040F22060C2F200000069002818BF80470B
:10204000A006A0D540F22060C2F20000406900283E
:1020500018BF8047600698D540F22060C2F20000A9
:102060008069002818BF8047200690D540F2206084
:10207000C2F20000C069002818BF8047E0057FF564
:1020800088AF40F22060C2F20000006A002818BF4A
:102090008047A0057FF580AF40F22060C2F20000CB
:1020A000406A002818BF804760057FF578AF40F28E
:1020B0002060C2F20000806A002818BF8047200517
:1020C0007FF570AF40F22060C2F20000C06A0028C5
:1020D00018BF8047E0047FF568AF40F22060C2F28D
:1020E0000000006B002818BF8047A0047FF560AF98
:1020F00040F22060C2F20000406B002818BF804709
:1021000060043FF557AF5DE710BD000043F6144192
:10211000C4F201010A6802421CBF0860FFF724BF35
:10212000704700002DE9F04F82B041F600420827C9
:1021300043F6004B4FF0010E002500244FF000083D
:10214000C4F20202C4F2010B904200F13E4202F1DD
:10215000FF7208BF07274FEAB223072B38BF4FEAA9
:10216000B22700970AE000BF08F1010804350234E5
:10217000B8F1100F04BF02B0BDE8F08F0E680EFA80
:1021800008FC16EA0C0FEFD0D1F8049009F0030A0E
:10219000AAF10106012E17D8D0F808E0CB68032277
:1021A00002FA04F62EEA0606A3404FF0010E33436E
:1021B0008360C9F30013466803FA08F326EA0C06A5
:1021C0003343436003E000BFBAF1030F23D0C66876
:1021D0000322BAF1020F02FA04F326EA03038E681F
:1021E00006FA04F643EA0603C36014D105F01C03A3
:1021F0000F2202FA03F64FF6FC72C7F6FF7202EAEC
:1022000058020244176AB7430E6906FA03F33B43C8
:102210001362D1F804900768032309F0030219F44C
:10222000403F03FA04F302FA04F227EA030342EA06
:102230000302026098D0002205F00C070F260192DD
:1022400043F64402BE40C4F2020213461A6842F446
:1022500080421A601A6802F48042019228F0030258
:10226000019B5A444FF60843CFF6FF73994652F844
:102270000930B343009E06FA07F73B4342F80930A2
:10228000DBF808204B6822EA0C0213F4801F18BF09
:1022900042EA0C0213F4001FCBF8082043F60C426C
:1022A000C4F201021646326822EA0C0218BF42EA62
:1022B0000C0213F4003F3260DBF8042022EA0C0227
:1022C00018BF42EA0C0213F4803FCBF80420DBF87D
:1022D000002022EA0C0218BF42EA0C02CBF80020D0
:1022E00042E70000002A08BF09048161704700002E
:1022F00040F20800C2F200008068704740F2080017
:10230000C2F20000017882681144816070470000C9
:1023100080B543F60040C4F20200016841F4007148
:102320000160016841F480610160016841F48071DD
:102330000160032000F08EF80F2000F005F800F097
:1023400025F8002080BD000070B540F20806044664
:102350004FF47A71C2F200063078B1FBF0F040F22F
:102360001401C2F200010968B1FBF0F000F07AFC40
:1023700001250F2C08D838B94FF0FF302146002234
:10238000002500F035F87460284670BD82B043F631
:10239000400100200190C4F202014A6842F48042E8
:1023A0004A604A6802F480420192019A00900868EB
:1023B000002240F08050086008680F2100F0805033
:1023C000009000986FF0010002B000F011B800001A
:1023D0000028B8BF704700F01F010122400902FA2F
:1023E00001F14EF20012CEF2000242F820107047C6
:1023F00010B500F00F034EF60C5E00F1604CB0F12A
:10240000FF3FA3F10403CEF2000E734403F10C046A
:10241000C8BF0CF56444DEF80000C0F3022000F1F0
:10242000040CC31E80F00700BCF1070F4FF0010C35
:1024300038BF0023042828BF04200CFA00F001381C
:1024400008400CFA03F10F31984011400843000195
:10245000207010BD4EF60C514FF6FF03CEF2000176
:102460000A681A4060F30A2242F0806040F0FD7072
:10247000086070472DE9F04104460D46002C00F03D
:10248000A78043F60808C4F20208D8F8F80300F061
:102490000700A84208D288F8F853D8F8F80300F0EB
:1024A0000700A84240F09480206810F0020F17D077
:1024B000410742BFD8F8001041F4E051C8F80010BD
:1024C000010742BFD8F8001041F46041C8F800107D
:1024D000D8F80010A26821F0F0011143C8F80010EC
:1024E000C00734D06068811E022905D258F8081C44
:1024F00011F0007F6CD00CE0012805D158F8081CC1
:1025000011F4003F64D004E058F8081C11F0020FE9
:102510005ED0D8F8001021F003010843C8F800008D
:10252000FFF7E6FE064641F2883700BFD8F8000004
:10253000616800F00C00B0EB810F08D0FFF7D8FE07
:10254000801BB842F2D90320C0B2BDE8F081D8F8B0
:10255000F80300F00700A84207D988F8F853D8F824
:10256000F80300F00700A84232D1206810F0040FF1
:1025700007D0D8F80010E26821F4E0511143C8F800
:102580000010000708D5D8F80000216920F4604049
:1025900040EAC100C8F8000000F046F8D8F8001082
:1025A00048F69422C0F60002C1F30311515CC84002
:1025B00040F21401C2F20001086040F20C00C2F2C5
:1025C00000000068FFF7C0FE0020C0B2BDE8F08147
:1025D0000120C0B2BDE8F08140F2140043F60801CA
:1025E00048F6A422C2F20000C4F20201C0F60002C2
:1025F00000680968C1F38221515CC840704700003F
:1026000040F2140043F6080148F6A422C2F200008A
:10261000C4F20201C0F6000200680968C1F3423149
:10262000515CC8407047000010B543F60404C4F282
:102630000204606800F00C0008280BD004281EBFBC
:1026400042F20040C0F2F40010BD41F60030C0F28A
:10265000B70010BD2268206841F600310023C0F2A7
:10266000B70110F4800F02F03F0204BF42F20041B4
:10267000C0F2F4012068C0F38810A1FB0001FDF74F
:102680009FFD21680222C1F3014102EB4101B0FB31
:10269000F1F010BD2DE9F04782B00446002C3FD088
:1026A000207843F6000A43F67007C4F2020AC4F227
:1026B0000207C0073FD057F8680C00F00C00042850
:1026C00030D057F8680C00F00C00082804D157F8F7
:1026D0006C0C10F4800F25D16668B6F5803F09D0E8
:1026E000DAF80000B6F5A02F40F0728140F48020A7
:1026F000CAF80000DAF8000040F48030CAF80000A0
:10270000FFF7F6FD054600BFDAF8000010F4003FC1
:1027100011D1FFF7EDFD401B6428F5D9032098E1A6
:10272000012096E1DAF8000010F4003F03D0606861
:10273000002800F0D480207840F20008C4F2472836
:10274000800737D557F8680C10F00C0F20D057F8D9
:10275000680C00F00C00082804BF57F86C0C10F44B
:10276000800F15D0E068002800F0A5800120C8F88F
:102770000000FFF7BDFD0546DAF8000010F0020F7B
:102780000FD1FFF7B5FD401B0228F5D9032060E10A
:10279000DAF8000010F0020F1CBFE068012840F0DA
:1027A0008880DAF80000216920F0F80040EAC100D2
:1027B000CAF800002078000725D5606988B101209B
:1027C000C8F8800EFFF794FD054600BF786810F04A
:1027D000020F18D1FFF78CFD401B0228F6D9032009
:1027E00037E10020C8F8800EFFF782FD054600BFE4
:1027F000786810F0020F06D0FFF77AFD401B022820
:10280000F6D9032025E12078400740F18C8057F865
:10281000300C4FF0000910F0805F0FD1CDF804901C
:102820004FF0010957F8300C40F0805047F8300C59
:1028300057F8300C00F080500190019843F60006E4
:10284000CFF6FE765AF8060010F4807F14D15AF8BD
:10285000060040F480704AF80600FFF749FD05467F
:102860005AF8060010F4807F06D1FFF741FD401BA7
:102870000228F5D90320ECE0A668012E05D03868BF
:10288000052E2ED140F004003860386840F0010079
:102890003860FFF72DFD054641F28836386810F0A4
:1028A000020F37D1FFF724FD401BB042F6D90320B9
:1028B000CFE00120CDE00020C8F80000FFF718FDB0
:1028C000054600BFDAF8000010F0020F3FF472AFC7
:1028D000FFF70EFD411B03200229F3D9B9E00120C7
:1028E000B7E020F001003860386820F0040038605C
:1028F000FFF7FEFC0546002ECED141F2883638683F
:1029000010F0020F06D0FFF7F3FC411B0320B14289
:10291000F5D99EE0B9F1010F02BF57F8300C20F055
:10292000805047F8300CA669002E00F0918057F8CF
:10293000680C00F00C00082803D1012E22D10120E0
:1029400087E00020C8F86000FFF7D2FC0546022EA1
:102950000CD100BFDAF8000010F0007F55D0FFF76F
:10296000C7FC411B03200229F4D972E0DAF8000009
:1029700010F0007F6CD0FFF7BBFC411B0320022945
:10298000F4D966E057F86C0CE16900F480028A42E1
:1029900063D1216A00F03F028A4260D1626A47F641
:1029A000C0710140B1EB821F5BD1A16A4FF6FF728B
:1029B000C903914300F44032A1F580318A4252D1DB
:1029C000E16A00F07060B0EB016F41D0012040E09F
:1029D00020F48030CAF80000DAF8000020F48020EB
:1029E000CAF80000FFF784FC0546002E7FF48CAE89
:1029F000DAF8000010F4003F3FF49DAEFFF778FCDA
:102A0000411B03206429F3D923E004F11C064FCEB7
:102A10000843D90340EA82104FF6FF72914340EA1F
:102A20000660A1F58031084347F86C0C0120C8F816
:102A30006000FFF75DFC0446DAF8000010F0007F4C
:102A400006D1FFF755FC011B03200229F4D900E051
:102A50000020C0B202B0BDE8F0870120F9E70120F4
:102A6000F7E70120F5E70120F3E7000070B5044621
:102A7000002C02BF0125284670BDD4F824C0BCF14B
:102A8000000F04D00021216104F1140105E0616808
:102A9000B1F5827F03D004F11C0100220A600025F9
:102AA0004FF0000EA56294F8511041B9204684F809
:102AB000505000F03FF8D4E909C101F4005E022251
:102AC00084F851202268136823F040031360D4E98E
:102AD0000130D4E9031603F4827300F4044001F4D6
:102AE00000611843084306F002010843616901F0E0
:102AF00001010843A16901F400731843E36903F07D
:102B000038031843236A03F08003184340EA0E0099
:102B10001060042000EA11400CF0100108435060DE
:102B2000D06920F40060D0610120656584F851000F
:102B3000284670BD2DE9F04786B00026044643F2D2
:102B400000070596CDE90366CDE90166C4F20107E9
:102B50002068B84202D006B0BDE8F08743F63000E6
:102B6000009601AD4FF002084FF003094FF0050A3F
:102B7000C4F20200416941F480514161416901F4AC
:102B80008051009100990096016841F002010160B6
:102B9000016801F00201009100990096016841F07E
:102BA000010101602946006800F0010000900098D2
:102BB0001820019007F55440CDE90286CDF8109019
:102BC000CDF814A0FFF7AEFA80202946CDE9010820
:102BD00003A880E8400607F55040FFF7A3FA40F24B
:102BE000900546F240474FF0C0694FF480684FF4BB
:102BF0004030C2F20005C4F20207C5E90079C5E918
:102C00000266C5E90486C5E90666C5E908062846E0
:102C1000FFF7A6F8002818BFFEF736FBE564AC63A3
:102C200040F2C03507F1180040210022C2F2000531
:102C3000C5E9000905F1080080E806014FF40030FD
:102C4000C5E90522EA61C5E908022846FFF788F8C8
:102C5000002818BFFEF718FBA564AC6306B0BDE8FA
:102C6000F0870000411E0020B0EB116F1CBF012057
:102C700070474EF21002F023CEF2000251604EF681
:102C80002351CEF200010B70072190601160704754
:102C9000704700007047000090F83C300222012B82
:102CA00055D010B5012380F83C3080F83D200268F3
:102CB000D2F804E0D2F808C00C682EF07003234369
:102CC000536041F2FF73C4F200039A42BDE8104022
:102CD0000BDC40F2FF73C4F200039A4213DCB2F142
:102CE000804F29D040F2004315E040F2FF33C4F298
:102CF00001039A4214DC41F60003C4F200039A4235
:102D00001AD0002314E040F60003C4F200039A42F4
:102D100012D040F60043C4F200039A420CD010E0F7
:102D200044F20003C4F201039A4205D040F200438A
:102D3000C4F201039A4204D149682CF0800319437C
:102D400091600121002280F83D1080F83C20D0B233
:102D50007047000010B50446002C04BF012010BDD0
:102D600094F83D0028B9002084F83C00204600F08B
:102D7000B1F8022040F6FF3284F83D00C4F20002B0
:102D80002068016890420FDCB0F1804F1EBF40F216
:102D90000043C4F20003984217D040F60003C4F287
:102DA0000003984211D014E040F60043C4F200033F
:102DB00098421EBF40F20043C4F20103984204D07F
:102DC0000023C4F20103984203D1A36821F07001EB
:102DD000194341F6FF73C4F2000398420DDC9042A0
:102DE0001FDCB0F1804F1EBF40F20042C4F200026F
:102DF00090423BD040F6000221E043F6FF72C4F25D
:102E00000102904220DC42F20002C4F20002904231
:102E10001EBF0022C4F20102904227D040F20042BD
:102E200020E040F60042C4F2000290421EBF41F68C
:102E30000002C4F20002904218D041F60042C4F2EF
:102E40000002904212D015E044F20002C4F20102E6
:102E500090421EBF44F60002C4F20102904205D027
:102E600044F20042C4F20102904203D1226921F4EB
:102E700040711143E268A36921F08001C2621943E5
:102E800040F200436268C4F20103826240F480624F
:102E90009A4204BF62690263026842F0040202605F
:102EA000012242610160002084F8462084F83E201F
:102EB00084F83F2084F8402084F8412084F84220A0
:102EC00084F8432084F8442084F8452084F83D2089
:102ED00010BD000080B584B0016844F2004243F6A2
:102EE0004000C4F20102C4F20200914218D041F243
:102EF0000042C4F2000291421FD040F60002C4F228
:102F00000002914217D100210391016841F00401B0
:102F10000160006800F004000390039804B080BDD5
:102F200000210191416841F400314160406800F4A2
:102F300000300190019804B080BD00210022029170
:102F4000016841F0200101600521006800F02000C7
:102F5000029002983720FFF74BFA372004B0BDE803
:102F60008040FFF735BA000090F83C300222012B78
:102F700000F0C58080B5012380F83C3080F83D200A
:102F80004FF67772D0F800C0DCF8083023EA02026E
:102F9000CCF808200B684F2B28DC1F2B43DD202B9F
:102FA00018BF302B43D0402B40F0AB80D1F804E069
:102FB000C968DCF82030DCF8202022F00102CCF8CF
:102FC0002020DCF8182022F0F00242EA0111CCF8AF
:102FD000181023F00A0141EA0E01CCF82010DCF8A9
:102FE000081021F0770141F047017DE06F2B26DDCD
:102FF000B3F5005F47D0B3F5805F77D0702B40F01A
:103000008080D1E90123C9681A4342EA0121DCF832
:10301000082022F47F421143CCF80810DCF8081095
:1030200041F0770160E0002B18BF102B69D1DCF86C
:10303000081021F07701194341F0070154E0502BAB
:1030400033D0602B5DD1D1F804E0C968DCF82030C2
:10305000DCF8202022F01002CCF82020DCF8182028
:1030600022F4704242EA0131CCF8181023F0A0019A
:1030700041EA0E11CCF82010DCF8081021F077019D
:1030800041F0670130E0D1E90123C9681A4342EAFF
:103090000121DCF8082022F47F421143CCF808100B
:1030A000DCF8081041F480411EE0D1F804E0C96862
:1030B000DCF82030DCF8202022F00102CCF82020BF
:1030C000DCF8182022F0F00242EA0111CCF81810C6
:1030D00023F00A0141EA0E01CCF82010DCF80810B8
:1030E00021F0770141F05701CCF8081000220121AE
:1030F00080F83D10002180F83C10BDE88040D0B23F
:1031000070470122F3E7000070470000B0B50446A5
:103110002068C168026901EA0205A90714D56FF0A9
:103120000201016101212177806910F0030F03D0B2
:103130002046FFF7E9FF05E0204600F075F820463D
:1031400000F04CFA00202077680715D520686FF052
:103150000401016102212177806910F4407F03D0CE
:103160002046FFF7D1FF05E0204600F05DF820463D
:1031700000F034FA00202077280715D520686FF07A
:103180000801016104212177C06910F0030F03D009
:103190002046FFF7B9FF05E0204600F045F820463D
:1031A00000F01CFA00202077E80615D520686FF0A3
:1031B0001001016108212177C06910F4407F03D01C
:1031C0002046FFF7A1FF05E0204600F02DF820463D
:1031D00000F004FA00202077E80706D020686FF09E
:1031E00001010161204600F0FBF9280606D52068A0
:1031F0006FF0800101612046FFF74AFD680606D5A1
:1032000020686FF040010161204600F0EBF9A8064C
:1032100058BFB0BD20686FF0200101612046BDE8B5
:10322000B040FFF737BD00007047000090F83C3019
:10323000012B02BF0223D8B270474FEAB20201232A
:10324000032A80F83C3000F201812DE9F041DFE8EB
:1032500002F002813EC303681E6A1A6A22F001026C
:1032600026F002061A621A46D3F804C052F8185F14
:103270008F680C68374325F0730643F4806546EA8F
:10328000040E40F20046C4F20106B54201BF27F029
:103290000C04CF6827F004072743B54201BFD1E9EA
:1032A00005452CF44076264346EA050CC3F804C0D5
:1032B000C3F818E04E685E631F629F6947F0080715
:1032C0009F619F6927F004079F610969B8E003685F
:1032D0001F6A1A6A22F4807227F400771A621A466B
:1032E000D3F804C052F81C4F8E680D6847EA062ECA
:1032F00040F2004624F0730444EA050843F4806574
:10330000C4F20106B54209D1CF6840F2FF443F0242
:1033100027EA04042EF4406744EA070EB54201BFD1
:10332000D1E905452CF4405747EA041747EA051C44
:10333000C3F804C0C3F81C804F68DF63C3F820E003
:10334000DF6947F00807DF61DF6927F00407DF6105
:10335000096975E003681F6A1A6A22F0100227F0F3
:1033600020071A621A46D3F804C052F8184F8E6824
:103370000D6847EA061E40F2004624F4E64444EA9B
:10338000052843F48065C4F20106B54201BFCF6849
:103390006FF04F0404EA07142EF0C00708BF44EA98
:1033A000070EB54201BFD1E905452CF4406747EA55
:1033B000840747EA850CC3F804C0C3F818804F6837
:1033C0009F63C3F820E09F6947F400679F619F698E
:1033D00027F480679F6131E00368D3F820C01A6A40
:1033E00022F480522CF400541A621A46D3F804E0F6
:1033F00052F81C6F8F680D6844EA073C26F4E644D7
:1034000040F2004644EA052543F48064C4F2010614
:10341000B44202BF4C692EF4804747EA841EC3F8C9
:1034200004E0DD614F681F64C3F820C0DF6947F422
:103430000067DF61DF6927F48067DF6109690902DE
:103440001368194300231160BDE8F041002180F8A2
:103450003C10D8B27047000010B50446002C04BFE1
:10346000012010BD94F83D0028B9002084F83C00EC
:10347000204600F0B1F8022040F6FF3284F83D000B
:10348000C4F200022068016890420FDCB0F1804F66
:103490001EBF40F20043C4F20003984217D040F62A
:1034A0000003C4F20003984211D014E040F6004338
:1034B000C4F2000398421EBF40F20043C4F201036D
:1034C000984204D00023C4F20103984203D1A368B8
:1034D00021F07001194341F6FF73C4F200039842D2
:1034E0000DDC90421FDCB0F1804F1EBF40F2004265
:1034F000C4F2000290423BD040F6000221E043F6C5
:10350000FF72C4F20102904220DC42F20002C4F2D7
:10351000000290421EBF0022C4F20102904227D056
:1035200040F2004220E040F60042C4F20002904225
:103530001EBF41F60002C4F20002904218D041F6CC
:103540000042C4F20002904212D015E044F20002A0
:10355000C4F2010290421EBF44F60002C4F201020E
:10356000904205D044F20042C4F20102904203D1DD
:10357000226921F440711143E268A36921F08001BE
:10358000C262194340F200436268C4F201038262DE
:1035900040F480629A4204BF62690263026842F0AA
:1035A00004020260012242610160002084F846208A
:1035B00084F83E2084F83F2084F8402084F841209D
:1035C00084F8422084F8432084F8442084F845207D
:1035D00084F83D2010BD00007047000070470000D7
:1035E000704700007047000070470000016844F613
:1035F00000020320C4F2000202F54C43994208BFC6
:103600000120914208BF0020032808BF7047C1B2C3
:10361000C90051FA80F040F26861C2F2000101EB8A
:103620008000006900B1004770470000F0B581B02C
:10363000044620680168C268456901F02F0602F05F
:103640002003202E06D12BB1204601B0BDE8F0406A
:1036500001F0A8BE5FEA017C08D005F0010E12F46B
:10366000907F8EF0010558D1002D56D01140CA062A
:10367000226B3CD5012A3AD10021009101680091CA
:10368000416800910099416911F0400F40F0D580E8
:10369000A18DE28DE38D002B00F04781891A89B25C
:1036A00009B942E1206850E8030F226820F49070C5
:1036B00042E80303002BF5D1206850E8050F22688B
:1036C00020F0010042E80503002BF5D1202084F80A
:1036D00042000020206300BF206850E8030F2268EA
:1036E00020F0100042E80303002BF5D107E10A06A1
:1036F00040F1EA8094F84110212940F01681A16838
:10370000B1F5805F04BF2169002900F00081216AC2
:103710004A1C22620978416000E1CE0706D012F40B
:1037200080761EBF666C46F00106666401F00407F1
:10373000012686EA97072F4302BF676C47F002070E
:10374000676401F0020786EA5706354302BF656CDD
:1037500045F00405656453EA0E0318BF0123BCF16C
:10376000000F05D5012B02BF636C43F008036364AF
:10377000636C002B00F0D9801140890603D52046E8
:1037800001F010FE20684169626C01F0400102F016
:103790000802114307D12046FFF728FF002060648C
:1037A00001B0F0BD206850E8030F216820F490704C
:1037B00041E80302002AF5D1206850E8050F21688E
:1037C00020F0010041E80502002AF5D1206B012814
:1037D0000AD100BF206850E8030F216820F01000D4
:1037E00041E80302002AF5D1202084F8420000209D
:1037F00020632068416911F0400F02D173E000BFDF
:10380000206850E8050F216820F0400041E80502DB
:10381000002AF5D1E06B002865D045F24921C0F6B9
:1038200000010165FEF7BCF9002800F07E80E06B26
:10383000016D01B0BDE8F0400847E36B19684D68C1
:10384000A28DA9B2002954D0914252D2E585D969FE
:10385000B1F5807F01D131E0206850E8030F216885
:1038600020F4807041E80302002AF5D1206850E876
:10387000050F216820F0010041E80502002AF5D17A
:10388000206850E8050F216820F0400041E805025B
:10389000002AF5D1202084F842000020206300BFD8
:1038A000206850E8030F216820F0100041E803026F
:1038B000002AF5D1E06BFEF731F9A28D022060639A
:1038C000E08D101A81B21CE049062ED5C16821F0A6
:1038D0004001C160202084F84100204601B0BDE8CD
:1038E000F04000F043BA204601B0BDE8F040FFF7D9
:1038F0007DBE8A4204BFD869B0F5807F15D1022011
:103900006063204601B0BDE8F040FFF76DBE216A5C
:1039100031F8022B6FF35F2242602162E18C4FF697
:10392000FF7201391142E18401D001B0F0BDC168DC
:1039300021F08001C160C16841F04001C16001B067
:10394000F0BD000010B50446002C04BF012010BDDE
:1039500094F8410028B9002084F84000204600F087
:1039600021F8242084F841002068C16821F4005126
:10397000C160204601F07CFD2068016921F490417E
:103980000161416921F02A014161C16841F400519E
:10399000C16000202021606484F8411084F8421046
:1039A000606310BD2DE9F04F87B00026044644F651
:1039B000000240F2000943F6300046F2280806965D
:1039C000CDE90466CDE90266C4F20002C4F2020940
:1039D000C4F20200C4F20208216891426ED041F2A2
:1039E0000042C4F20102914200F0B38041F20002B1
:1039F000C4F20102914240F01281002702AE4FF062
:103A0000020A4FF0030B07250197416941F01001AD
:103A10004161416901F0100101910199019701682B
:103A200041F002010160016801F002010191019978
:103A30000197016841F0010101603146006800F022
:103A40000100019001988020029009F58060CDE985
:103A500003A7CDF814B00695FEF764FB4FF4007091
:103A60003146CDE9020A4846CDE9047B0695FEF7CA
:103A700059FB40F2F00508F58C604FF000614FF4FF
:103A80008062C2F2000585E883004FF44030C5E94A
:103A90000372C5E90577EF61C5E908072846FEF717
:103AA0005FF9002818BFFDF7EFFB25200521002254
:103AB000E563AC63FEF79CFC252045E001960169B7
:103AC00041F480210161016901F480210191019992
:103AD0000196016841F00401016002A9006800F04C
:103AE0000400019001984FF4406002900220CDE95B
:103AF0000306032005900720069009F50060FEF7F5
:103B000011FB40F220454FF000604FF48061C2F29B
:103B10000005C5E900804FF40030C5E90266C5E93B
:103B20000416C5E90666C5E908062846FEF718F931
:103B3000002818BFFDF7A8FB272005210022E56318
:103B4000AC63FEF755FC2720FEF742FC07B0BDE84A
:103B5000F08F00260196416941F0200141614169E1
:103B600001F02001019101990196016841F04001A5
:103B7000016002A9006800F04000019001984FF434
:103B8000844002900220CDE903060320059008201E
:103B9000069009F5C050FEF7C5FA40F2105508F539
:103BA00080604FF0206A4FF480694FF48037C2F292
:103BB0000005C5E9000A2846C5E90266C5E904967C
:103BC000C5E90666C5E90876FEF7CAF8002818BFF9
:103BD000FDF75AFBE563AC6340F2C05508F58F6012
:103BE0004021C2F20005C5E9000A05F1080080E89D
:103BF00042022846C5E90566EE61C5E90876FEF78A
:103C0000AFF8002818BFFDF73FFB47200521002231
:103C1000A563AC63FEF7ECFB4720FEF7D9FB07B0CA
:103C2000BDE8F08FB0B582B0044613460A4694F85A
:103C3000420020282BD1002A4FF0010018BF002B92
:103C400026D00025222045F2013145F28D3C256326
:103C5000A262A385656484F84200C0F60001C0F644
:103C6000000CE06BC0E90F1C45F25521C0F60001C5
:103C7000C0E9131521680431FEF724F900280AD0A1
:103C800010206064202084F84200012000E002201F
:103C9000C0B202B0B0BD01952068016801914168D1
:103CA00001910199216911B90AE000BF206850E82B
:103CB000030F216840F4807041E80302002AF5D127
:103CC000206850E8050F216840F0010041E8050236
:103CD000002AF5D1206850E8050F216840F0400027
:103CE00041E80502002AF5D10020D1E7016844F639
:103CF00000020320C4F2000202F54C43994208BFBF
:103D00000120914208BF0020032808BF7047C1B2BC
:103D1000C90051FA80F040F26861C2F2000101EB83
:103D20008000C06800B1004770470000016844F699
:103D300000020320C4F2000202F54C43994208BF7E
:103D40000120914208BF0020032808BF7047C1B27C
:103D5000C90051FA80F040F26861C2F2000101EB43
:103D60008000806800B1004770470000016844F699
:103D700000020320C4F2000202F54C43994208BF3E
:103D80000120914208BF0020032808BF7047C1B23C
:103D9000C90051FA80F040F26861C2F2000101EB03
:103DA0008000406800B1004770470000FEE7000057
:103DB000002804BF9FED150A704790ED011A90EDA1
:103DC000066A90ED022A90ED077AF0EE400A90ED37
:103DD000033A90ED044A90ED055A46EE410A47EE4B
:103DE000420A10EE901A21F00041B1F1FF4F08BFD6
:103DF000F0EE400A23EE200AC0ED060A80ED076AC5
:103E000006EE040A07EE050A704700BF0000000036
:103E100010B50446002C08BF10BDF5EEC00A002006
:103E2000C4ED000AF1EE10FAC4E9060028DD9FEDAA
:103E3000201A80EE200A81EE000A04F083FC9FED38
:103E40001D1AB7EE002ABFEE003A20EE011A20EE4E
:103E5000000A31EE024A32EE411A30EE032A30EE09
:103E6000044A30EE011A32EE022A80EE040A81EE94
:103E7000043A82EE044A30EE001AB0EE402A09E01D
:103E80009FED0A1AB7EE000AB0EE412AB0EE414AA1
:103E9000B0EE413A84ED014A84ED023A84ED030A22
:103EA00084ED041A84ED052A10BD00BF0000000057
:103EB000DB0F4940F304B53F002804BF9FED1B0A08
:103EC000704790ED033A90ED044A90ED055A90ED5D
:103ED000011A90ED022AB0EE407A33EE046A36EE13
:103EE000056A80EE066A16EE101A01F0FF41B1F184
:103EF000FF4F18BFB0EE467AB0EE406A01EE476A57
:103F000002EE476A16EE101A21F00041B1F1FF4FA0
:103F100008BFB0EE406A23EE060A80ED066A80ED27
:103F2000077A07EE040A07EE050A70470000000052
:103F30000146002902BFFE2040B2704708780128E0
:103F400032D840F2B062C2F2000252F820205AB3D6
:103F50004988A1F201210A296FD880B584B00123D4
:103F600003FA01F10B0722D111F0F00F3CD040F21F
:103F7000FF11009108218DF8041051890B0A8DF86A
:103F800005308DF8061091890B0A8DF807308DF8F1
:103F90000810D1890B0A8DF809308DF80A10118AA2
:103FA0000A0A8DF80B203AE0FC2040B270474FF42B
:103FB0000071009108218DF80410D1788DF805105A
:103FC00091788DF8061051798DF8071011798DF8D8
:103FD0000810D1798DF8091091798DF80A10517A6D
:103FE0008DF80B10117A1AE040F2FF2100910821A0
:103FF0008DF80410518A0B0A8DF805308DF80610E3
:10400000918A0B0A8DF807308DF80810D18A0A0AB8
:104010008DF809208DF80A1000218DF80B108DF80D
:104020000C106946FCF77CFC002818BF4FF0FF30ED
:1040300004B0BDE8804040B27047FF2040B27047F6
:1040400010B500B3017801291DD840F2B062C2F268
:10405000000252F8211000291CBF91F844E0BEF183
:10406000000F10D001F1180C002300BF5CF82310E2
:1040700019B142884C88944203D001337345F5DB73
:104080000021084610BD0021084610BDF0B581B0E2
:10409000044624B12678012E05D9FF2000E0FE2039
:1040A00040B201B0F0BD40F2B067C2F2000757F86D
:1040B0002600B8B157F8266036B396F8440028B306
:1040C00006F11801002200BF51F822301BB16788A9
:1040D0005B88BB4238D001328242F5DB0A2815D911
:1040E000FF20DDE74820FCF72DFC0546002D47F8B2
:1040F000265027D028464821FCF7BFF82E70267896
:10410000012ED7D9FF20CBE7FF20C9E75020FCF7CD
:1041100019FC0546D5B1206861686960286005F121
:1041200018002821FCF7A9F86079032285F82800F7
:1041300061882078FCF7F0FA50B12846FCF700FCC3
:10414000FF20ADE7FF20ABE7FD20A9E7FF20A7E7B1
:1041500096F8440006EB8000856196F84400013033
:1041600086F8440000209BE710B5002802BFFE201F
:1041700040B210BD0178012934D840F2B062C2F2D9
:10418000000252F821C0BCF1000F2BD0B7EE001A8C
:10419000BFEE002AB4EEC10AF1EE10FAC8BFB0EECD
:1041A000410A41799CF844E0B4EEC20AF1EE10FAFB
:1041B000B8BFB0EE420AB1EE401A002908BFB0EE17
:1041C000401ABEF1000F0DD00CF11801002200BF03
:1041D00051F822301BB15B884488A34205D00132DC
:1041E0007245F5DBFC2040B210BD0079022805D2F3
:1041F000A3F2012189B2072906D31EE01DD1A3F243
:10420000052189B2052918D848F6882140B2C0F6A0
:10421000000101EB800090ED000A4FF07F4000EBC1
:1042200003600CEBE05021EE000ABDEEC00A10EE78
:10423000101A4180002040B210BDFF2040B210BDD6
:10424000F0B587B0024622B11078012803D9FC20CE
:104250001DE0FE201BE040F2B061C2F2000151F807
:10426000201089B191F8443083B101F11804002580
:1042700054F825701FB179885688B1420AD00135AB
:104280009D42F5DBFC2002E0FC2000E0FC2040B277
:1042900007B0F0BD6A460023FCF7F8F978B1FCF7E7
:1042A00053FBD7E90823801A40F2E9329941801A7A
:1042B00071F1000028D300203876FC20E7E70120C8
:1042C0003876FCF741FBC7E908019DF811009DF81D
:1042D000121097F904509DF80E309DF80F209DF8AC
:1042E000106041EA00219DF80D0046EA0222022DED
:1042F00043EA00200AD84FA64BA306EB850653F8E5
:10430000253096ED004A05E0FF20C0E7B7EE004AF1
:104310004FF0FF339FED4A1A09B200EE100A12B2B5
:104320009FED483A5943B8EEC05A06EE102A9FED69
:10433000460A02EE101AB8EEC22A25EE015AB8EE6D
:10434000C61AB97922EE032A25EE003A41B1B7F830
:104350004010411AB1F5805F08DD4FF0FF3109E0F0
:1043600000217964A7F84000B96418E011F5805F76
:1043700004DA01217A6C1144796400E0796C05EE6D
:10438000101A81EE041A24EE022AB8EEC55AA7F8D4
:10439000400005EE003A83EE043A87ED123A87EDCD
:1043A000023A87ED031A87ED042A97F8280048B3EC
:1043B000B5EEC03AF1EE10FA08DA33EE003AB5EE97
:1043C000C03AF1EE10FAF8DB87ED023AB4EEC03AEB
:1043D000F1EE10FA0ADB9FED1D4A33EE043AB4EE1B
:1043E000C03AF1EE10FAF8DA87ED023A30EE430AFD
:1043F000B1EE411AB1EE422A87ED020A87ED031AA7
:1044000087ED042A9DF8130007F1080307F12C0C2F
:1044100000EE100AB8EE400A87ED050A0FCB8CE8D3
:104420000F00002033E700BF10270000004000000D
:104430003075000000001042000098410000803FED
:104440000000003900008038DB0FC940DB0FC9C015
:1044500080B540F6A41046F200414FF4A022C2F20B
:104460000000C4F200010160032141600021C0E9A5
:10447000021102614FF4C002426181838161FDF744
:10448000B1F800281CBFBDE88040FCF7FDBE80BD30
:1044900080B540F6CC1046F600014FF4C022C2F2BF
:1044A0000000C4F200010160032141600021C0E965
:1044B000021102614FF4A002426181838161FDF724
:1044C00091F800281CBFBDE88040FCF7DDBE80BD30
:1044D00080B582B043F6300100200190C4F20201A1
:1044E0000A6842F400120A600A6802F4001201929B
:1044F000019A00900868002240F480000860086873
:10450000052100F48000009000980C20FDF770FF5A
:104510000C20FDF75DFF392005210022FDF768FF23
:104520003920FDF755FF3A2005210022FDF760FFF5
:104530003A20FDF74DFF3B2005210022FDF758FFF3
:104540003B20FDF745FF442005210022FDF750FFE9
:104550004420FDF73DFF452005210022FDF748FFDF
:10456000452002B0BDE88040FDF732BF80B544F67B
:10457000057048F620320021C0F60000C0F60002A7
:1045800001F04EFB40F6A01148F6AC22C2F2000149
:10459000C0F60002086044F6F1700021C0F6000089
:1045A000BDE8804001F03CBB2DE9F04786B043F602
:1045B00030000026002400224FF4E05A05960096B1
:1045C000C4F20200C4F20204016804F5E05741F0AD
:1045D00002010160016801F002010091009900965A
:1045E000016841F040010160016801F04001009163
:1045F00000990096016841F001010160016801F035
:104600000101009100990096016841F008010160E4
:10461000016801F00801009100990096016841F0DD
:1046200004010160016801F0040100910099009605
:10463000016841F080010160016801F08001009192
:1046400000990096016841F0200101604FF4E051AB
:10465000006800F02000009000983846FDF742FE08
:104660002046102101224FF010090125FDF73AFEE6
:1046700004F58068012101224046FDF733FECDE9B3
:1046800001A50396022001AE049038463146FDF79D
:1046900049FD4FF48817204631460195CDE9027552
:1046A000FDF740FD20463146CDE90195CDE90355A2
:1046B000FDF738FD30203146CDE9010704F50060F3
:1046C0000395FDF72FFD40463146CDE90155CDE973
:1046D0000355FDF727FD062005210022FDF788FE82
:1046E0000620FDF775FE0A2005210022FDF780FE59
:1046F0000A20FDF76DFE172005210022FDF778FE48
:104700001720FDF765FE06B0BDE8F08710B540F64E
:10471000F41043F200014FF4827200234FF0010CB9
:104720004FF4007E1824C2F20000C4F2010180E8B8
:104730000E000A21C0E90333C0E905CEC461C0E917
:104740000833C0E90A31FEF791F900281CBFBDE823
:104750001040FCF799BD10BD70B58EB040F64C20EE
:1047600044F20045002141F28732C2F20000C4F257
:1047700001050791CDE90511CDE90311CDE901113D
:10478000C0E90051C0E9021201618161FEF7E2FA5D
:10479000002818BFFCF778FD40F64C20C2F200005C
:1047A000FEF75AFE002818BFFCF76EFD40F64C24B9
:1047B0006020002601A90022C2F200040190CDE988
:1047C000026605962046FEF731FD002818BFFCF76B
:1047D0005BFD0D96CDE90B66CDE9096643F6300029
:1047E0002168C4F20200A9421FD040F60002C4F2C0
:1047F0000002914231D100210891026842F0080282
:104800000260006800F00800089008984FF48040AB
:1048100009900220CDE90A01CDE90C1005F54840C8
:1048200009A9FDF77FFC0EB070BD00210891026858
:1048300042F020020260006800F020000890089812
:10484000402009900220CDE90A010C90032009A91B
:104850000D9005F55040FDF765FC0EB070BD0000F1
:10486000B0B594B040F6942040F60005002145F222
:104870000722C2F20000C4F200050D91CDE90B1130
:10488000CDE90911CDE90711CDE90511CDE90311F4
:10489000CDE90111C0E90051C0E902120161816155
:1048A000FEF758FA002818BFFCF7EEFC4FF48050D2
:1048B0000AA90A9040F69420C2F20000FEF754FBC9
:1048C000002818BFFCF7E0FC40F69420C2F200007C
:1048D000FEF7C2FD002818BFFCF7D6FC40F6942076
:1048E000002408A9C2F20000CDE90844FEF7D4F97B
:1048F000002818BFFCF7C8FC602001A90822CDE9F8
:1049000001040394059440F69424C2F20004204666
:10491000FEF78CFC002818BFFCF7B6FC002044F220
:10492000004343F630011390CDE91100CDE90F00AB
:10493000C4F20103C4F2020122689A421BD0AA42C7
:1049400030D100200E900A6842F008020A6009681F
:1049500001F008010E910E994FF480410F91022150
:10496000CDE91010CDE9120105F501300FA9FDF7D1
:10497000D9FB14B0B0BD0E900A6842F020020A6064
:10498000096801F020010E910E9940210F9102213A
:10499000CDE91010032012910FA9139005F50330F3
:1049A000FDF7C0FB14B0B0BD10B582B040F6DC20FE
:1049B00041F20041002440F2473240F2E733C2F2B4
:1049C0000000C4F20001CDE9004480E81600C36095
:1049D0008461FEF7BFF9002818BFFCF755FC40F6CC
:1049E000DC206946CDE90044C2F20000FEF754F92C
:1049F000002818BFFCF748FC02B010BD80B540F697
:104A0000243041F200014FF4E13200234FF00C0C4E
:104A1000C2F20000C4F2010180E80E00C0E90333D5
:104A2000C0E905C3C361FEF78DFF00281CBFBDE8C8
:104A30008040FCF729BC80BD80B540F66C3044F660
:104A4000000C48F2A0624FF4805300214FF00C0E8E
:104A5000C2F20000C4F2000CC0F20102C0E900C2C0
:104A6000C0E90231C0E9041EC0E90611FEF76AFF81
:104A700000281CBFBDE88040FCF706BC80BD0000DC
:104A800080B540F6B43041F200414FF4E1320023EA
:104A90004FF00C0CC2F20000C4F2010180E80E00DD
:104AA000C0E90333C0E905C3C361FEF74BFF00282B
:104AB0001CBFBDE88040FCF7E7BB80BDFEE70000FF
:104AC000F0B581B02DED048BB0EE408A1446A8B14C
:104AD0000078052816D8DFE800F01985990303A5AA
:104AE000012B0DDB00200022002100BF013144F822
:104AF0002200CAB29342F9DCFF206EE0FF206CE096
:104B0000FF206AE0012B35DA002066E0042BE7D1B4
:104B100091ED000A91ED011A91ED022A30EE410A61
:104B200030EE020A84ED000A91ED000A91ED011ABF
:104B300091ED022A30EE010A30EE020A84ED010AFC
:104B400091ED000A91ED011A91ED022A31EE400A31
:104B500030EE020A84ED020A91ED000A91ED011A8D
:104B600091ED022AB1EE400A30EE410A30EE020A1F
:104B700084ED030A9FED2E9ADDB227462E4600BF34
:104B800097ED000A03F043FCB4EEC90A013E043776
:104B9000F1EE10FAC8BFB0EE409A002EF0D1B7EE99
:104BA000000AB4EEC09AF1EE10FA0BDD2846214659
:104BB00091ED000A013880EE090A81ED000A01F149
:104BC0000401F5D194ED000A013D20EE080A84EDC0
:104BD000000A04F10404F5D1002040B2BDEC048BBE
:104BE00001B0F0BD042B7FF47BAF91ED000AB1EE74
:104BF000400A84ED000A086860600868A06091EDD2
:104C0000000AB1EE400A84ED030A6BE7022B7FF441
:104C100067AF91ED000AB1EE400A84ED000A086822
:104C200060605FE7012B7FF45BAF0868206059E7A5
:104C30000000000000280EBFFF200170002040B2DD
:104C400070470000FEE70000B0B52DED0A8B04466A
:104C500010EE100AB0EE618AB0EE419AB0EE60BA82
:104C600000F0FF40B0F1FF4F00F09B801BEE100AF8
:104C700000F0FF40B0F1FF4F00F0938019EE100AF2
:104C800000F0FF40B0F1FF4F00F08B8018EE100AEB
:104C900000F0FF40B0F1FF4F00F083806068F0EE5D
:104CA0004B0A90ED071AFCF76DF96068B0EE40AA68
:104CB00090ED001A04F11C0021EE0B0A2AEE01CA45
:104CC000FFF776F82078B0EE40BA70B101280ED127
:104CD00094ED050AD4ED020A3BEE409AB0EE480A84
:104CE00003F044FC89EE009A01E09FED309A84EDD8
:104CF00004AA84ED05BA19EE100A9FED2C0A656826
:104D000094ED03AA00F0FF40B0F1FF4F0CEE08AAAB
:104D100095ED022A9FED268A95ED011A95ED033A4D
:104D200018BFB0EE490A2CEE019AB4EEC82A2AEE5A
:104D300002BA00EE439AF1EE10FA1EDD1AEE100AE6
:104D400000F0FF40B0F1FF4F17D039EE0B0A03F02F
:104D50005EFB95ED051AB4EEC10AF1EE10FA0CDC1B
:104D6000B0EE4A0A03F053FB95ED041AB4EEC10A03
:104D7000F1EE10FAD8BF84ED03AA39EE0B0A10EE5B
:104D8000100A00F0FF40B0F1FF4F0AD0D5ED050A40
:104D9000F4EEC80AF1EE10FAC8BFFBF761FC84ED2F
:104DA000060A94ED060ABDEC0A8BB0BD00000000B7
:104DB000BD37863570B504460D464CB3506800F0DB
:104DC000FF40B0F1FF4F23D0906800F0FF40B0F1FA
:104DD000FF4F1DD0D06800F0FF40B0F1FF4F17D05B
:104DE000106900F0FF40B0F1FF4F11D0506900F0A2
:104DF000FF40B0F1FF4F0BD0B7EE001A626081EEBA
:104E0000001A11EE100A00F0FF40B0F1FF4F02D17E
:104E1000FF2568B270BD84ED021A04F11C06D2EDC4
:104E2000060A3046FEF7F4FF9FED060A25700025BE
:104E30003046C4E90355C4E90555FFF73DF868B2AB
:104E400070BD00BF0000000010B5002802BFFF24A5
:104E500060B210BD9FED050A0024C0E90344C0E91B
:104E600005441C30FFF728F860B210BD00000000B8
:104E7000EFF30980BFF36F8F154B1A681EF0100F08
:104E800008BF20ED108A20E9F04F10602DE90900DD
:104E90004FF0500080F31188BFF34F8FBFF36F8F37
:104EA00002F0FAF84FF0000080F31188BDE8090025
:104EB00019680868B0E8F04F1EF0100F08BFB0EC9A
:104EC000108A80F30988BFF36F8F704700BF00BF5F
:104ED000A80C0020000000000000000000000000FE
:104EE000074B19680868B0E8F04F80F30988BFF3F2
:104EF0006F8F4FF0000080F31188704700BF00BF34
:104F0000A80C002080B500F089FEBDE8804000F0CC
:104F1000D7BE000080B5FDF7F1F902F08FFF012840
:104F20001CBFBDE8804002F08FB980BDB0B592B023
:104F300043F6400000240225CDE90A44CDE90844A7
:104F40000594CDE90344CDE901440094C4F2020084
:104F5000016841F080510160006800F080500090CD
:104F60000098009447F20000C4F20000016841F488
:104F700080410160006800F48040009000980120AA
:104F800006904FF4803007904FF480000C950D9000
:104F900006200E904820CDE90F050420119006A8A8
:104FA000FDF778FB08B172B6FEE70F200221CDE9CC
:104FB00001054FF480500394CDE9040401A8FDF7E6
:104FC00059FA002804BF12B0B0BD72B6FEE7000067
:104FD0004EF68850CEF20000016841F47001016085
:104FE0007047000040F6DC20C2F20000FEF78EB8E9
:104FF00010B500F0FDFB45F2710048F6D02200210B
:10500000C0F60000C0F6000200F00AFE41F20C14E7
:1050100048F6F4220021C2F20004C0F6000220602B
:1050200045F29910C0F6000000F0FAFD6060022021
:105030000A21002200F074FCA06002205821002206
:1050400000F06EFCE06002201021002200F068FCFD
:10505000206102201821002200F062FC606100F053
:10506000FDFB00F0DBFDBDE8104000F029BE0000B4
:105070002DE9F04F81B02DED028B00F09FFB07462C
:105080000020002400F066FB00F090FB0546FBF7D3
:10509000A3FFFBF7A1FF9FED3E0A40F2B86940F67F
:1050A000FC320146C2F20009C2F200024846FBF798
:1050B00037FE9FED358B40F220363846C2F20006AF
:1050C00034707460FBF7B2F953EC182BB460FBF743
:1050D000DFF8F460FBF7B7F941F20C1840F2B04B7F
:1050E000074606F1100A3D44C2F20008C2F2000B66
:1050F00019E000BFD8F8100031460022002300F06C
:10510000CFFB48465946FBF7F9FE00F04FFB02463D
:1051100048463146FBF794FC4846FBF7C3FE284659
:1051200000F028FB3D44D8F814005146002200232B
:1051300000F0B6FB0028DDD1BE4606F11007A446FC
:105140008FCF746A8BE88F00CBF8144006F11007FC
:105150008FCF746AC9F88C02C9F89012C9F89422EA
:10516000C9F89832C9F89C72C9F8A0425FEACC70BD
:105170004FF0010406D1F06940F6FC310124C2F27F
:10518000000108607746B5E70000000000407F405E
:105190000000FA43000000002DE9F04700F00EFB8C
:1051A0000446002000F0D6FA2046FBF73FF99FEDB9
:1051B000240B53EC102BFBF76BF8FBF744F9044678
:1051C00000F0F4FA40F250364FF6F87841F20C1A3B
:1051D00005194FF40139C2F20006C0F2FF08C2F20D
:1051E000000A06F110070AE0DAF810003146002242
:1051F000002300F0D5FB284600F0BCFA25443846D1
:10520000FCF718F81420FCF725F8012814D13846CB
:10521000FBF71AFF96F84900411E002002299CBFA7
:1052200008EAC10029FA00F03070B06B7060706B52
:10523000B060F06BF060D7E73846FBF7F7FED3E7D6
:105240000000000000407F40806B0021C185FEF718
:10525000CDB90000806B01684A6990F84130212B7C
:1052600014D112F0800211D00022C28401E000BFEC
:10527000016851E8031F026821F0C00142E80313EE
:10528000002BF5D1202180F8411001684A6990F87F
:105290004230222B2DD112F040022AD00022C285AA
:1052A00001E000BF016851E8031F026821F490711A
:1052B00042E80313002BF5D1016851E8051F02688D
:1052C00021F0010142E80513002BF5D1016B012902
:1052D0000AD100BF016851E8031F026821F01001E4
:1052E00042E80313002BF5D1202180F84210002161
:1052F0000163416C41F010014164FEF777B9000091
:105300000168806B096811F4807F32D10021C1856A
:10531000016851E8031F026821F4807142E8031319
:10532000002BF5D1016851E8051F026821F0010149
:1053300042E80513002BF5D1016851E8051F02680A
:1053400021F0400142E80513002BF5D120218446CD
:1053500080F842105CF8302F012A0CD1026852E824
:10536000032F036822F0100243E803210029F5D13E
:1053700001E000F1300C00214163DCF8001001294C
:1053800018BFFEF7B3BC818DFEF72EB9806B0121EB
:105390004163016B012918BFFEF7C8BC818D490824
:1053A000FEF722B990F84210222918BF704783688F
:1053B000B3F5805F06D1026900F12801A2B1D1F8EE
:1053C00000C008E00146002B51F828CF01D1036945
:1053D0000BB17F2300E0FF23026852681A400123CB
:1053E0008CF800200A6806E00368826A5B686FF345
:1053F0005F23138002231A440A604FF6FF72C18DA7
:1054000001391142C18500D070470168CA6822F095
:105410002002CA60CA6822F48072CA604A6922F017
:1054200001024A61202280F8422000224263036B7D
:10543000012B18BFFEF75ABC026300BF51E8031FDF
:10544000026821F0100142E803130168002BF5D136
:105450000A6812F0100F08D081B0002200920A688A
:10546000009249680091009901B0818DFEF7BCB8A7
:10547000B0B5044649F20C6520680169E26821F480
:10548000405111430161D4F808C0D4E90423D4F891
:105490001CE0C16842EA0C02A9431A4342EA0E0228
:1054A0001143C1604169A26921F440711143416116
:1054B00041F2004140F48060C4F20101884202D10F
:1054C000FDF79EF801E0FDF787F8E26963681921AE
:1054D000A0FB0101B2F5004F1CD15A00DB0FFAF717
:1054E0006FFE48F21F51C5F2EB11A0FB01235A09D0
:1054F0006FF0630302FB0300322303EBC000A0FB49
:1055000001014FF4F87000EA1110C1F3421100EBF1
:1055100002101AE09A009B0FFAF752FE48F21F5150
:10552000C5F2EB11A0FB01235A096FF0630302FBE4
:105530000300322303EB0010A0FB0101F02000EA7E
:105540005110C1F3431100EB021008432168886039
:10555000B0BD000040F62430C2F20000FEF766B88D
:1055600010B582B040F66C30C2F2000000680168ED
:1055700011F0200F3BD144F60001C4F2000109688C
:1055800011F0100F55D0002141F248130091C2F2E2
:1055900000030168009140680090009840F22040AC
:1055A000C2F2000000680268016821F0010112F4F3
:1055B000002F01604168C1F1320119804FF03203C0
:1055C00043601DD1026842F400220260026842F08A
:1055D0000102026088B219282BD140F2C020C2F229
:1055E0000000283002B0BDE8104000F0EDBF0021FF
:1055F00001910168019140680190019802B010BDCD
:1056000046F22802C4F20202136823F40023136056
:10561000026842F00102026088B2192809D140F202
:10562000C024C2F2000404F1410000F0CDFF0120CB
:10563000207002B010BD000010B540F6B434C2F2C4
:1056400000042046FDF7F2FF2046BDE81040FBF7BE
:10565000B3B90000FEE700002DE9F04104466CB349
:1056600040F6A840C2F200000068A04202BF00203D
:10567000C0B2BDE8F08101F059F940F250186569F7
:10568000C2F20008D8F81860D8F81C7001F074F95C
:10569000B5424FF0020018BFBD420CD008F14C00DB
:1056A000854214D00120002D08F1380108BF0420E4
:1056B0008D4208BF0420C0B2BDE8F0814FF0500019
:1056C00080F31188BFF36F8FBFF34F8FFEE7A06A9F
:1056D00000281EBF0220C0B2BDE8F08194F8581027
:1056E0000320012908BF0220C0B2BDE8F0810000FC
:1056F00080B5FCF70DFEFFF719FCFEF755FFFEF72E
:10570000E7FEFEF7A5FEFEF7C3FEFFF795F9FFF7EC
:10571000B7F9FEF7FBFFFFF771F9FFF7A1F8FFF705
:1057200043F9FFF719F800F04DF8FEF71FFF00F0FE
:1057300075F800BFFEE7000032EE612A30EE600A25
:1057400031EE601A20EE020A80EE010A30EE210AE4
:1057500070470000EFF3058100291CBF6FF00500C2
:105760007047002804BF0020704780B501F01CFA84
:10577000002080BD10B582B00446EFF305800028FC
:105780001EBF6FF0050002B010BD02F067FB211ACA
:1057900001900129BEBF6FF0030002B010BD01A847
:1057A00001F04CFA002002B010BD0000EFF30580BC
:1057B000002808BF02F052BB02F056BB4FF47A70CB
:1057C00070470000EFF3058000281CBF6FF0050054
:1057D000704740F26460C2F20000016800291CBFFB
:1057E0004FF0FF307047012101600020704700003A
:1057F00080B5EFF3058010B16FF0050080BD02F0B9
:105800001DFB002804BF012080BD02281CBF4FF0F3
:10581000FF3080BD01F038FC002080BD10B5EFF3F3
:10582000058000281EBF6FF00504204610BD40F221
:105830006460C2F20000016801291EBF4FF0FF340E
:10584000204610BD4EF61F510024CEF200010C7010
:105850000221016001F0D2FB204610BD10B5EFF32C
:10586000058000281EBF6FF00504204610BD02F021
:10587000E5FA022802BF0024204610BD60B902F0FC
:10588000DDFC0124012809D002F0D8FA002808BF65
:105890004FF0FF34204610BD4FF0FF34204610BDBE
:1058A00010B582B0B1FA81F21C46B0FA80F3520909
:1058B0005B091A43EFF30583EBB1002C18BF0124F9
:1058C000224319D10022019201AA02F027F80128EF
:1058D0001EBF6FF0020002B010BD0198A8B14EF6D5
:1058E00004504FF08051CEF200000160BFF34F8FA3
:1058F000BFF36F8F09E01AB16FF0030002B010BD63
:10590000224601F03DFF012802D1002002B010BD67
:105910006FF00100002C08BF6FF0020002B010BD54
:10592000B0B582B000291446EFF305824FF00005B0
:1059300018BF002830D07ABB04B3D4E9023273B167
:10594000502A0FD322699AB1D4F814E001FB00FC6D
:105950000025E64520D3009501F0D4FC11E01AB1F2
:10596000002519E0002517E022691AB1002513E08F
:10597000002511E062690AB100250DE0002201F066
:105980007BFC05463DB1002C284614BF2168002150
:1059900001F0ACF800E00025284602B0B0BD0000E0
:1059A000B0B582B0B1FA81F21D46B0FA80F3520967
:1059B0005B091A43EFF305833BB1002D18BF0125A6
:1059C0002A4306D06FF003042CE0CAB16FF0030441
:1059D00028E000220023019201AA01F009FE01281B
:1059E0001CD10198E8B14EF604504FF080510024CC
:1059F000CEF200000160BFF34F8FBFF36F8F11E055
:105A00002A460023002401F0EDFC01280AD06FF0A3
:105A10000104002D08BF6FF0020403E06FF00204E0
:105A200000E00024204602B0B0BD000010B50C46D6
:105A30000146EFF3058010B16FF0050010BD21F0B5
:105A40000100002804BF6FF0030010BD11F0010138
:105A500007D1214601F0BEFF012804BF002010BD80
:105A600006E0214602F098F8012804BF002010BD8E
:105A70006FF00100002C08BF6FF0020010BD0000A5
:105A800080B50146EFF3058000281CBF6FF00500CC
:105A900080BD21F00100002804BF6FF0030080BD2D
:105AA00011F001010BD100210022002301F09AFC2A
:105AB0006FF00201012808BF0021084680BD01F0F7
:105AC0003DFE01466FF00200012908BF002080BDA5
:105AD0002DE9F04F81B08146EFF3058017460C4663
:105AE00028B16FF0050B584601B0BDE8F08FB9F151
:105AF000000F15DB14F0020F4E466FF0010B18BFBC
:105B00000026002F08BF6FF0020B02F0A7F98046B5
:105B100014F0010F07D1002F47D00025EA4619E005
:105B20006FF0030BDFE7002F5AD00024EA4625E090
:105B300002F094F9A0EB08003F1A38BF002709E0F3
:105B4000009904EA090041EA000515EA090FEFD0BF
:105B500061E000BF0020314652463B462C4602F031
:105B60001DFA0028BFD001285D46F3D1E8E702F016
:105B700075F9A0EB08003F1A38BF00270020314616
:105B800052463B46254602F009FA0028ABD00128D0
:105B90005C46F3D1009905EA090041EA000404EAF1
:105BA00009004845E3D1A3469DE700206C4600BFAD
:105BB0000546002031462246002302F0EFF9002876
:105BC0003FF491AF01285846F2D1009905EA090047
:105BD00041EA000B1BEA090F08BF6FF0020B82E7D6
:105BE00000206C460546002031462246002302F084
:105BF000D5F900283FF477AF01285846F2D1009933
:105C000005EA090041EA000B0BEA0900484518BF04
:105C10006FF0020B67E7AB4665E7000002F008B9DA
:105C2000F0B585B000238C4600280493EFF305817E
:105C30003BD0D1BB42B19469002C08BF1824611E2F
:105C4000372911D9002330E000218023182404AA29
:105C5000CDE900429AB2634602F002F801281ABF69
:105C600000230493049B20E01179C9071CD111681B
:105C7000D2E9025756694FEA960E002E734608BFC6
:105C80008023ADB100235C2F0FD3002E1CBF1269FF
:105C9000002A0AD0CDE9004272466346029502F01E
:105CA0004DF80346049300E00023184605B0F0BD0C
:105CB0000FB10023F9E71269002AC8D00023F4E7E6
:105CC00010B50446EFF3058000281CBF6FF00500F7
:105CD00010BD64B12046FFF7BFFC042804BF6FF07D
:105CE000020010BD204601F01BF8002010BD6FF02F
:105CF000030010BD2DE9F041044600F017FE40F20C
:105D0000501740F6A848C2F20007C2F20008B8686F
:105D10000130B860D8F8000060B1F868002840F0A1
:105D20000C81D8F80000E16AC06A884298BFC8F8C0
:105D3000004002E1C8F80040B868012840F0FD804A
:105D400040F6AC45C2F20005284600F0ABFD05F177
:105D5000140000F0A7FD05F1280000F0A3FD05F1F7
:105D60003C0000F09FFD05F1500000F09BFD05F1A7
:105D7000640000F097FD05F1780000F093FD05F157
:105D80008C0000F08FFD05F1A00000F08BFD05F107
:105D9000B40000F087FD05F1C80000F083FD05F1B7
:105DA000DC0000F07FFD05F1F00000F07BFD05F563
:105DB000827000F077FD05F58C7000F073FD05F53D
:105DC000967000F06FFD05F5A07000F06BFD05F515
:105DD000AA7000F067FD05F5B47000F063FD05F5ED
:105DE000BE7000F05FFD05F5C87000F05BFD05F5C5
:105DF000D27000F057FD05F5DC7000F053FD05F59D
:105E0000E67000F04FFD05F5F07000F04BFD05F574
:105E1000FA7000F047FD05F5027000F043FD05F54E
:105E2000077000F03FFD05F50C7000F03BFD05F537
:105E3000117000F037FD05F5167000F033FD05F523
:105E40001B7000F02FFD05F5207000F02BFD05F50F
:105E5000257000F027FD05F52A7000F023FD05F5FB
:105E60002F7000F01FFD05F5347000F01BFD05F5E7
:105E7000397000F017FD05F53E7000F013FD05F5D3
:105E8000437000F00FFD05F5487000F00BFD05F5BF
:105E90004D7000F007FD05F5527000F003FD05F5AB
:105EA000577000F0FFFC05F55C7000F0FBFC05F599
:105EB000617000F0F7FC05F5667000F0F3FC05F585
:105EC0006B7000F0EFFC05F5707000F0EBFC05F571
:105ED000757000F0E7FC05F57A7000F0E3FC05F55D
:105EE0007F7000F0DFFC05F5826000F0DBFC05F25E
:105EF000244000F0D7FC05F5876000F0D3FC05F2E4
:105F00004C4000F0CFFC40F28045C2F2000528462C
:105F100000F0C8FC05F11406304600F0C3FC07F1A0
:105F2000600000F0BFFC07F1380000F0BBFC07F197
:105F30004C0000F0B7FCBD61FE613868013038608C
:105F40006064E06A396A884240F6AC4188BF3862D2
:105F500000EB8000C2F2000101EB8000211D00F087
:105F6000CFFC00F009FDF86890B1D8F80000E16AB4
:105F7000C06A884228BFBDE8F0814EF604504FF059
:105F80008051CEF200000160BFF34F8FBFF36F8FDF
:105F9000BDE8F0812DE9F04140F2501540F6AC46E5
:105FA0004EF604584FF08057C2F20005C2F20006C8
:105FB000CEF2000803E000BF204600F0F5FC686860
:105FC000D0B100F0B3FC686CC468201D00F03CFC4C
:105FD000A8680138A86068680138686000F0CCFCE7
:105FE00094F8590020B10128E6D00228E7D00DE04E
:105FF000206B00F0D9FCDFE730680228DFD3C8F857
:106000000070BFF34F8FBFF36F8FD8E74FF0500092
:1060100080F31188BFF36F8FBFF34F8FFEE700004F
:1060200008480068006880F308884FF0000080F39B
:10603000148862B661B6BFF34F8FBFF36F8F00DF76
:1060400000BF00BF08ED00E02DE9F04F85B08146AC
:1060500001F004FF40F2D0148346C2F2000420692C
:10606000834538D2A068016881B34FF0000A0DF172
:10607000040800BFC068C76805683E1D304600F0D0
:10608000E3FB396A3846884797F82800400719D556
:10609000B8692844A84207D978603F613146A068B2
:1060A00000F010FC0EE000BF2068E8B1CDE901A5CA
:1060B000039701F0C3FE206841460022002301F04F
:1060C00091F988B1A06801680029D3D1E168C4E9D9
:1060D0000210012000E00020C9F80000C4F810B050
:1060E000584605B0BDE8F08F4FF0500080F311889E
:1060F000BFF36F8FBFF34F8FFEE7000081B000202A
:10610000009040F28800C2F2000000684FF0500199
:1061100081F31188BFF36F8FBFF34F8F013001D030
:10612000FEE700BF00980028FCD001B070470000D7
:106130002DE9F04F89B040F2D01601AC4FF00009C4
:106140000DF11408EA46C2F2000600BFB0684FF035
:10615000000B0768002F1CBFC068D0F800B000F02B
:1061600093FF2046FFF770FF0546019810B102F03B
:1061700065F84DE0AFB15D4513D302F05FF8B0684C
:10618000C068C76807F10409484600F05DFB97F84E
:10619000280010F0040F1FD100F0FE0087F828003F
:1061A0002CE0002227B9F0680068B0FA80F04209BC
:1061B0003068ABEB050100F0D3FC02F03FF838BBD0
:1061C0004EF604504FF08051CEF200000160BFF354
:1061D0004F8FBFF36F8F1BE0B86900EB0B01A94233
:1061E00079603F6101D9B06805E0A5EB0B01814200
:1061F00080F08C80F068494600F064FB4FF00009A5
:10620000396A3846884703E000F0FE0087F8280026
:1062100030682146002201F0B3FA002896D0019898
:10622000B0F1FF3F06DCDDE90220049990470198B8
:106230000028EDDB039F786900281CBF381D00F0A3
:1062400003FB5046FFF700FF01990929E0D8DFE87A
:1062500001F0050505373A530505373A97F8281038
:1062600041F0010187F82810391DBD69029AAB1869
:1062700083427B603F6104D9904235D2934203D27E
:1062800032E0801AA84233D3396A3846884797F8F3
:1062900028004007BCD53268B8690299002A50D05E
:1062A0000844CDF81490CDE9060701F0C7FD306829
:1062B00041460022002301F095F80028A8D140E0D3
:1062C00097F82800A0E797F8281041F0010187F817
:1062D000281002990029B9613DD00A18394641F8C1
:1062E000042F82423F6103D9B06800F0EBFA8FE7D8
:1062F000F06800F0E7FA8BE797F8280010F0020F3B
:106300007FF482AF384600F04FFB81E7306878B108
:106310004FF00009CDE9059B079701F08FFD30682C
:1063200041460022002301F05DF800287FF468AFA9
:106330004FF0500080F31188BFF36F8FBFF34F8F82
:10634000FEE74FF0500080F31188BFF36F8FBFF36B
:106350004F8F00BFFEE74FF0500080F31188BFF36E
:106360006F8FBFF34F8F00BFFEE70000F0B581B025
:10637000044600F0DBFA94F94560012E10DB04F1CD
:10638000240500BF286858B1284601F015FF0028F1
:1063900018BF00F043FD71B2701E01290646F1DC02
:1063A000FF2684F8456000F0E7FA00F0BFFA94F9A0
:1063B0004470012F10DB04F1100500BF286858B1AC
:1063C000284601F0F9FE002818BF00F027FD79B239
:1063D000781E01290746F1DC84F8446001B0BDE86D
:1063E000F04000F0C9BA000070B5044600F04CFE61
:1063F00040F21020C2F20000016849B145F6144194
:10640000C2F200010978002918BF4FF000412AE0CC
:1064100041F65C160025C2F20006F31D16F00702D5
:10642000314623F0070318BF19469B1B4FF47056E3
:10643000002AC0E9051518BFC3F570568A19083A35
:1064400022F007020260C2E90055521A4A6003684E
:106450000B6045F61441C0E901220122C2F200019D
:106460000A704FF000410025002C00F07D80214093
:106470007AD104F1080313F007010ED0C1F108012D
:106480000B4413F0070F08D04FF0500080F3118831
:10649000BFF36F8FBFF34F8FFEE741685A1E8A42EA
:1064A00021D2064656F8142F3146164675689D428D
:1064B00002D23268002AF7D10268964213D03268BD
:1064C000D1F800E00A60E91A112933D3F51815F064
:1064D000070F0AD04FF0500080F31188BFF36F8F81
:1064E000BFF34F8FFEE700253EE06960736000F167
:1064F000140300BF1C462368AB42FBD361686218DB
:10650000AA4202D0D5F804C005E06A68254602EB2D
:10651000010CC4F804C005EB0C01994206D10168D6
:106520008B421FBF5968614469601B68AC422B6095
:1065300018BF2560716842680EF10805521A426062
:1065400083689A4238BF826045F61442C2F2000264
:106550001278002A4FF0000218BF41F00041C6E94E
:106560000021C1680131C16001F068FE680704BF05
:10657000284670BD4FF0500080F31188BFF36F8F35
:10658000BFF34F8FFEE7000040F6A840C2F20000C4
:10659000016800291FBF01680A6D01320A650068A1
:1065A0007047000046F2FD0321F001014FF0807CAE
:1065B000C0F6000340E903316FF0020140F804CC5B
:1065C00040E9091244387047002808BF70472DE998
:1065D000F0412DED048B4178827840F2C0244FF4D5
:1065E000C066DFED910A9FED911ABFEE008AB7EE0B
:1065F000009AC2F20004F0EE481AB0EE492A62F3A3
:106600000A2100EE101AB8EEC00A84ED010A817862
:10661000C278C90862F34A1100EE101A4FF4806183
:10662000B8EEC00A84ED020AC278037947799B006C
:1066300001EA872743EA92123A4300EE102AB8EEA5
:10664000C00A84ED030A42798379520863F3CA12BF
:1066500000EE102AB8EEC00A84ED040A8279C379EC
:10666000120963F30A12A282C279037A477A5B00A5
:1066700006EA472743EAD2123A43E282427A837A11
:10668000920863F38A122283827AC37ADB0043EA98
:1066900052126283027B437B63F30A22A283427B12
:1066A000837BD20863F34A12E283827BC37B077C3D
:1066B0009B0001EA872143EA921211432184017C65
:1066C000407C490860F3CA11618494ED020AFFF727
:1066D00033F8B1EE400ADFED560A9FED561AF0EEA0
:1066E000481AB0EE492A84ED020A94ED010AFFF738
:1066F00023F884ED010ADFED500A9FED501AF0EE09
:10670000481AB0EE492A94ED030AFFF715F8B1EEE6
:10671000400ADFED4B0A9FED4B1AF0EE481AB0EE3F
:10672000492A84ED030A94ED040AFFF705F8B0EE58
:10673000408A84ED048A6068F9F79EFE9FED320B73
:1067400006460F4658EC105B2A464346F9F70FFE03
:1067500058B99FED2F0B3046394653EC102BF9F703
:1067600021FE002804BF00206060A068F9F784FEC5
:106770002A46434606460F46F9F7F9FD58B99FEDFC
:10678000240B3046394653EC102BF9F726FE00282F
:1067900004BF0020A060E068F9F76EFE9FED1E0BBD
:1067A00006460F4653EC102BF9F7E1FD58B99FED63
:1067B0001C0B3046394653EC102BF9F70EFE00281F
:1067C00004BF0020E06018EE100AF9F755FE2A46D3
:1067D000434606460F46F9F7CAFD58B99FED0C0B24
:1067E0003046394653EC102BF9F7F7FD002804BF6B
:1067F0000020206101202070BDEC048BBDE8F04139
:10680000704700BF00BF00BF7B14AE47E17A84BF72
:106810007B14AE47E17A843F9A9999999999A9BFD7
:106820009A9999999999A93F00007C4300E0CC443A
:106830000000994300A0D3440000944200C0B1443A
:10684000000042430080C544D0E9013201699A60EA
:10685000826853604B68834208BF4A60002202612D
:1068600008680138086008687047000045F25C73EA
:10687000C2F20003036045F25C50C2F200000860FF
:10688000802010607047000045F6B833C2F2000364
:10689000036045F2B870C2F2000008604FF48070E7
:1068A0001060704700F108014FF0FF32C0E901129B
:1068B000C0E903110021016070470000002101615F
:1068C0007047000080B5D1F800C01CF1010208D06B
:1068D00000F108029646DEF8042013686345F9D9F2
:1068E00003E0D0F810E0DEF804204A609160C1F8BF
:1068F00008E0CEF80410086101680131016080BD34
:1069000042684A6093688B6093685960916008613F
:106910000168013101607047DFF80C00016841F443
:1069200070010160704700BF88ED00E04FF050003B
:1069300080F31188BFF36F8FBFF34F8F40F2880051
:10694000C2F2000001684A1C0029026000D07047B2
:106950004EF60450CEF20000006810F0FF0F08BFA2
:1069600070474FF0500080F31188BFF36F8FBFF373
:106970004F8F00BFFEE7000040F28800C2F2000027
:10698000016839B10139016018BF7047002080F3F8
:10699000118870474FF0500080F31188BFF36F8F5C
:1069A000BFF34F8FFEE70000B0B50446002C08BFD0
:1069B000B0BD45F6144154F8040CA4F10805C2F228
:1069C00000010978002918BF4FF0004101420AD0A8
:1069D0002A6892B14FF0500080F31188BFF36F8F97
:1069E000BFF34F8FFEE74FF0500080F31188BFF3E5
:1069F0006F8FBFF34F8F00BFFEE7884344F8040C4E
:106A000000F042FB40F2102C54F8043CC2F2000C9F
:106A1000DCF804100CF114021944CCF8041000BF87
:106A200011460A68AA42FBD34C680819A84202BF63
:106A300023444B600D46E818904207D1DCF8000073
:106A400082421FBF5068184468601268A9422A60D9
:106A500018BF0D60DCF810000130CCF81000BDE864
:106A6000B04001F0EBBB00004EF210000021CEF26E
:106A700000000160816041F63F11C0F201014160F8
:106A80000721016070470000EFF30580102814D340
:106A90004EF2F031CEF20001405C40F22C21C2F205
:106AA00000010978884208D24FF0500080F3118825
:106AB000BFF36F8FBFF34F8FFEE74EF60C5040F2DF
:106AC0002C21CEF20000C2F200010068496800F4F7
:106AD000E060884298BF70474FF0500080F3118803
:106AE000BFF36F8FBFF34F8FFEE7000045F6184CE2
:106AF000C2F2000CDCF80020FAB1634653F8082F0C
:106B0000F2B1634653F8102FE2B1634653F8182FE1
:106B1000D2B1634653F8202FC2B1634653F8282FF1
:106B2000B2B1634653F8302FA2B1634653F8382F01
:106B3000002A18BF704707220DE0002263460AE0D2
:106B4000012208E0022206E0032204E0042202E01F
:106B5000052200E0062219600CEBC2014860704774
:106B600070B515460E460446FFF7E0FE94F8440063
:106B7000FF2804BF002084F8440094F84500FF2853
:106B800004BF002084F84500FFF7F6FEA06B28B98B
:106B900004F1240031462A4600F08EF92046BDE873
:106BA0007040FFF7E3BB0000F0B581B00446C4B30A
:106BB00040F25015C2F20005286940B14FF0500074
:106BC00080F31188BFF36F8FBFF34F8FFEE7286903
:106BD00040F6A846C2F20006013028616F693068AD
:106BE0000430FFF731FE30683C44BC4244604FF053
:106BF000010028BF0020002805D0E8693168043171
:106C0000FFF760FE08E0A86931680431FFF75AFE1B
:106C1000A86A844238BFAC6201F010FB08B101B031
:106C2000F0BD4EF604504FF08051CEF200000160EE
:106C3000BFF34F8FBFF36F8F01B0F0BD88B1D1B1FB
:106C40002DE9F04140F25014C2F200042269E2B191
:106C50004FF0500080F31188BFF36F8FBFF34F8F59
:106C6000FEE74FF0500080F31188BFF36F8FBFF342
:106C70004F8F00BFFEE74FF0500080F31188BFF345
:106C80006F8FBFF34F8F00BFFEE722690132226191
:106C9000666902685518964202D2954202D320E0F6
:106CA000954201D3B5421CD940F6A8480560C2F20E
:106CB00000086769D8F800000430FFF7C5FDA81B7D
:106CC0003D18D8F80000BD4245604FF0010028BFD4
:106CD000002040B1E069D8F800100431FFF7F2FD60
:106CE0000BE0056009E0A069D8F800100431FFF757
:106CF000E9FDA06A854238BFA56201F09FFA00282D
:106D0000BDE8F04118BF70474EF604504FF0805177
:106D1000CEF200000160BFF34F8FBFF36F8F70475B
:106D2000F0B581B00446FFF701FE002C02BF40F62B
:106D3000A840C2F200000468251D2846FFF784FD24
:106D4000A06A00281CBF04F11800FFF77DFD40F287
:106D5000501640F6A847C2F20006C2F2000730689B
:106D6000013030603868844217D0B0680138B060B4
:106D700094F85900022808D0012803D068BB206B82
:106D8000FFF712FE2046FFF70FFEB069006868B1FA
:106D9000B069C068C06840680AE006F1380029465A
:106DA000FFF7AEFD70680130706002E04FF0FF3019
:106DB000B062FFF7E1FDF06810B13868844201D09D
:106DC00001B0F0BD306990B14FF0500080F31188F0
:106DD000BFF36F8FBFF34F8FFEE74FF0500080F38C
:106DE0001188BFF36F8FBFF34F8F00BFFEE74EF6E2
:106DF00004504FF08051CEF200000160BFF34F8F7E
:106E0000BFF36F8F01B0F0BD40F25011C2F200012C
:106E10004A6B0260496941607047000040F25010BF
:106E20000121C2F20000C16270470000F0B581B0DC
:106E30000C4618B340F6A846C2F200063168183175
:106E4000FFF740FD40F25015C2F200056F6930684F
:106E50000430FFF7F9FC601C19D030683C44BC4298
:106E600044604FF0010028BF0020C8B1E8693168D4
:106E7000043101B0BDE8F040FFF724BD4FF05000F1
:106E800080F31188BFF36F8FBFF34F8FFEE7316838
:106E900005F14C00043101B0BDE8F040FFF730BD12
:106EA000A86931680431FFF70DFDA86A844238BF34
:106EB000AC6201B0F0BD00002DE9F04115460C4672
:106EC00000B340F6A847C2F2000739681831FFF74F
:106ED00017FD40F25018C2F20008D8F81460386864
:106EE0000430FFF7B1FC002D18BF4FF0FF3412D073
:106EF000601C10D1396808F14C000431BDE8F04144
:106F0000FFF7FEBC4FF0500080F31188BFF36F8F86
:106F1000BFF34F8FFEE738683444B44244604FF00B
:106F2000010028BF002038B1D8F81C0039680431AE
:106F3000BDE8F041FFF7C6BCD8F818003968043145
:106F4000FFF7C0FCD8F82800844238BFC8F82840B2
:106F5000BDE8F08170B5044624B3226D1AB3E06C2D
:106F6000884238BF0846012A1CD1E16A814208BF25
:106F700070BD40F6A842C2F200021268A2421CD0C4
:106F8000E06240F6AC46A269C2F20006002AA4BF45
:106F9000C0F13800A06101EB8100616906EB80005F
:106FA000814214D070BD4FF0500080F31188BFF3C0
:106FB0006F8FBFF34F8F00BFFEE74FF0500080F39D
:106FC0001188BFF36F8FBFF34F8F00BFFEE7251D02
:106FD0002846FFF739FC40F25011E06AC2F2000186
:106FE0000A6A904288BF086200EB8000294606EBDF
:106FF0008000BDE87040FFF783BC000010B586B08C
:10700000002405A804A903AACDE90444FFF72EFC37
:10701000DDE9032005990023CDE9004045F6957090
:10702000029117A1C0F6000000F088FE40F2501453
:107030000028C2F20004606216D001F079F9411C08
:1070400014D0012810D14FF0500080F31188BFF305
:107050006F8FBFF34F8F4FF0FF30A0620120E060D1
:107060000020606100F05EF806B010BD4FF05000E7
:1070700080F31188BFF36F8FBFF34F8FFEE700BF20
:1070800049444C450000000040F25010C2F200009C
:10709000016901310161704780B540F2501EC2F2B2
:1070A000000EDEF8101000291EBF0121CEF82C10B2
:1070B00080BD002140F6AC4CCEF82C10C2F2000C82
:1070C000DEF8201001EB81035CF8232052B90CEBB1
:1070D0008302A2F1140300BFD1B153F8142901397E
:1070E000002AF9D001EB81020CEB820353F8042F44
:1070F0005268181D1A60824204BF52681A60D06834
:1071000040F6A842C2F200021060CEF8201080BD06
:107110004FF0500080F31188BFF36F8FBFF34F8F94
:10712000FEE700004EF200404CF27021CEF200006B
:10713000C4F20F11D0F800294B1C9A4209D14FF02C
:10714000500080F31188BFF36F8FBFF34F8F00BFE4
:10715000FEE7D0F800298A4209D14FF0500080F3B1
:107160001188BFF36F8FBFF34F8F00BFFEE7B0B53D
:1071700084B001780291FF21017001788DF8071029
:107180009DF8071001F0500240F22C21C2F20001DC
:107190000A7007224A609DF90720B2F1FF3F49DCDF
:1071A000062200BF4A60013A9DF807305B008DF867
:1071B00007309DF90730002BF4DB022A3AD14FF457
:1071C00040724A6002990170D0F8201941F47001B0
:1071D000C0F82019D0F8201941F07041C0F82019EA
:1071E000FFF742FC40F288040025C2F2000425604B
:1071F000FFF792FB4EF63470CEF20000016841F0CA
:1072000040410160FEF70CFFFFF746FF0395206841
:107210004FF0500181F31188BFF36F8FBFF34F8F91
:10722000013001D0FEE700BF03980028FCD0002009
:1072300004B0B0BD4FF0500080F31188BFF36F8FE2
:10724000BFF34F8FFEE7000080B54FF0500080F392
:107250001188BFF36F8FBFF34F8F00F00FFE002830
:107260001FBF4EF60450CEF200004FF08051016077
:10727000002080F3118880BD2DE9F04107461446B7
:107280000E46A7B306FB07F05030FFF7ADF80546F2
:1072900055B34FF00008002E284685F8468018BFE9
:1072A00050302860C5E90F76FFF740FB2868D5E924
:1072B0000F1202FB01030139AB60C5F8388068602A
:1072C00001FB0200E860FF2085F8440085F84500D6
:1072D00005F11000FFF7E6FA05F12400FFF7E2FAE6
:1072E000FFF74AFB85F84C402846BDE8F0814FF097
:1072F000500080F31188BFF36F8FBFF34F8F00BF33
:10730000FEE70000B0B582B01C4660B1ACB1F1B987
:10731000EAB14FF0500080F31188BFF36F8FBFF3D5
:107320004F8F00BFFEE74FF0500080F31188BFF38E
:107330006F8FBFF34F8F00BFFEE74FF0500080F319
:107340001188BFF36F8FBFF34F8F00BFFEE751B1BE
:107350004AB94FF0500080F31188BFF36F8FBFF32D
:107360004F8F00BFFEE75023069D0193019B502BDA
:107370002DD1019B00294FF0010384F8463008BF4E
:1073800022462260C4E90F01FFF7D0FA2068D4E951
:107390000F1202FB01030139A3600023A3636060A5
:1073A00001FB0200E060FF2084F8440084F84500FF
:1073B00004F11000FFF776FA04F12400FFF772FAE7
:1073C000FFF7DAFA84F84C50204602B0B0BD4FF017
:1073D000500080F31188BFF36F8FBFF34F8F00BF52
:1073E000FEE700002DE9F04F83B0044617461D4626
:1073F0000E46002C029714D0EEB1022D03D1E06BA3
:10740000012840F0A38000F019FD00BBFFB14FF050
:10741000500080F31188BFF36F8FBFF34F8F00BF11
:10742000FEE74FF0500080F31188BFF36F8FBFF37A
:107430004F8F00BFFEE7206C0028DED04FF05000D9
:1074400080F31188BFF36F8FBFF34F8FFEE7FFF715
:107450006DFAA06B022D5AD0E16B884257D304F12C
:1074600010086F464FF0000A0298002800F07F8055
:10747000BAF1000F04D13846FFF7C6FC4FF0010AFD
:10748000FFF77AFAFFF700FEFFF750FA94F844008E
:10749000FF2804BF002084F8440094F84500FF282A
:1074A00004BF002084F84500FFF766FA384602A9B9
:1074B00000F092FB00285DD1FFF738FAD4F838B01D
:1074C000D4F83C90FFF758FACB4515D102994046C5
:1074D000FFF7ACFC2046FEF749FF00F0AFFE80B995
:1074E0004EF604504FF08051CEF200000160BFF321
:1074F0004F8FBFF36F8F04E02046FEF737FF00F099
:107500009DFEFFF713FAA06BE16B8842ACD2A76B2C
:10751000226C22B3BDB3E0683146F8F795FEE1680E
:10752000206C091AE160226891423FBF4042A16885
:107530000844E060002FA5F102013846B1FA81F15C
:1075400018BF0120490908403F1A29E04FF05000B8
:1075500080F31188BFF36F8FBFF34F8FFEE7206872
:107560000025E8B9A06800F091FDA56019E0FFF7DB
:1075700003FA04E02046FEF7F9FE00F05FFE00206B
:1075800003B0BDE8F08F60683146F8F75DFE6068D3
:10759000216C08446060A168884224BF2068606054
:1075A0000020791CA16354F8241F79B1204600F013
:1075B00003FEB8B14EF604514FF08050CEF20001F8
:1075C0000860BFF34F8FBFF36F8F0BE050B14EF6E3
:1075D00004514FF08050CEF200010860BFF34F8F8E
:1075E000BFF36F8FFFF7C8F9012003B0BDE8F08F3C
:1075F0002DE9F04705461E4614460F46E5B127B370
:10760000022E02D1E86B012852D1FFF73DFAEFF3C9
:1076100011884FF0500080F31188BFF36F8FBFF3D4
:107620004F8F022EA86B1CD0E96B884219D388F3C8
:1076300011880020BDE8F0874FF0500080F31188DA
:10764000BFF36F8FBFF34F8FFEE7286C0028D7D0B2
:107650004FF0500080F31188BFF36F8FBFF34F8F4F
:10766000FEE795F84590A86BD5F838A02A6C002A5B
:1076700027D0002E2DD0E8683946F8F7E5FDE968F7
:10768000286C091AE9602A6891423FBF4042A96804
:107690000844E860BAF1000FA6F102015046B1FAC1
:1076A00081F118BF012049090840AAEB000A1DE03A
:1076B0004FF0500080F31188BFF36F8FBFF34F8FEF
:1076C000FEE7286890B9A86800F0E0FC0020A860F8
:1076D0000CE068683946F8F7B7FD6868296C08441B
:1076E0006860A968884224BF286868600AF10100C0
:1076F000B9F1FF0FA86308D009F1010085F8450032
:10770000012088F31188BDE8F08755F8240F78B17F
:10771000284600F051FD0146002C4FF0010018BF33
:107720000029EED00120206088F31188BDE8F087A1
:1077300088F311880120BDE8F0870000B0B5044649
:10774000A4B1A56800F074FB85421CBF0020B0BD49
:10775000E0680138E0601CBF0120B0BD2046002178
:1077600000220023FFF73EFE0120B0BD4FF0500085
:1077700080F31188BFF36F8FBFF34F8FFEE70000D8
:107780002DE9F04F85B0044616460D46002C0496B0
:107790000FD0002D46D000F051FBA0B99EB14FF0A4
:1077A000500080F31188BFF36F8FBFF34F8F00BF7E
:1077B000FEE74FF0500080F31188BFF36F8FBFF3E7
:1077C0004F8F00BFFEE7FFF7B1F8D4F83890B9F15A
:1077D000000F34D0226C52B1E0688118E160A068DB
:1077E0008142284624BF2168E160F8F72DFDA9F108
:1077F0000100A06354F8100F70B1204600F0DCFCCB
:1078000050B14EF604514FF08050CEF200010860A6
:10781000BFF34F8FBFF36F8FFFF7AEF8012005B0B6
:10782000BDE8F08F206C0028B5D04FF0500080F3F9
:107830001188BFF36F8FBFF34F8F00BFFEE7002E9D
:1078400065D004F124004FF0000A02AF0DF11008DA
:107850004FF0000B019000BFBBF1000F04D1384680
:10786000FFF7D2FA4FF0010BFFF786F8FFF70CFC99
:10787000FFF75CF894F84400FF2808BF84F844A0A0
:1078800094F84500FF2808BF84F845A0FFF774F876
:107890003846414600F0A0F960B12046FEF766FD8B
:1078A00000F0CCFCFFF742F8A66BFFF765F81EBBB3
:1078B0002FE000BFFFF73AF8A66BFFF75DF82EB197
:1078C0002046FEF753FD00F0B9FC15E0049901983D
:1078D000FFF7ACFA2046FEF749FD00F0AFFC58B9BF
:1078E0004EF604504FF08051CEF200000160BFF31D
:1078F0004F8FBFF36F8F00BFFFF718F8D4F83890A1
:10790000B9F1000F7FF466AF04980028A4D1FFF707
:1079100033F8002005B0BDE8F08F00002DE9F043FA
:1079200081B0054691460E4635B376B3FFF7ACF805
:10793000EFF311884FF0500080F31188BFF36F8F81
:10794000BFF34F8FAC6B64B395F844702A6C52B19F
:10795000E8688118E960A8688142304624BF296838
:10796000E960F8F771FC601EFF2FA8631BD0781C3C
:1079700085F84400012028E04FF0500080F3118882
:10798000BFF36F8FBFF34F8FFEE7286C0028CDD079
:107990004FF0500080F31188BFF36F8FBFF34F8F0C
:1079A000FEE7002011E055F8100F68B1284600F0FE
:1079B00003FC01460120B9F1000F06D000291CBFCD
:1079C0000120C9F8000000E0012088F3118801B00F
:1079D000BDE8F0832DE9F04F85B004460D46002C3C
:1079E00004950AD0206C90B14FF0500080F31188BC
:1079F000BFF36F8FBFF34F8FFEE74FF0500080F360
:107A00001188BFF36F8FBFF34F8F00BFFEE700F009
:107A100015FA50B94DB14FF0500080F31188BFF303
:107A20006F8FBFF34F8F00BFFEE7FEF77FFFA06BA6
:107A3000F0B10138A063206810B9FEF7A5FDA06081
:107A400054F8100F70B1204600F0B6FB50B14EF65E
:107A500004514FF08050CEF200010860BFF34F8F09
:107A6000BFF36F8FFEF788FF012005B0BDE8F08FF0
:107A700004F124004FF0000902AE04AF4FF0000BF8
:107A80004FF0000A019061E0BBF1000F04D13046D5
:107A9000FFF7BAF94FF0010BFEF76EFFFFF7F4FAAC
:107AA000FEF744FF94F84400FF2808BF84F8449090
:107AB00094F84500FF2808BF84F84590FEF75CFF66
:107AC0003046394600F088F860B12046FEF74EFC9B
:107AD00000F0B4FBFEF72AFFA56BFEF74DFF7DB962
:107AE00043E000BFFEF722FFD4F83880FEF744FFE2
:107AF000B8F1000F09D02046FEF738FC00F09EFBDD
:107B0000FEF714FFA06B08B393E7206838B9FEF7BF
:107B10000DFFA06800F006FB8246FEF72DFF0499DA
:107B20000198FFF783F92046FEF720FC00F086FB62
:107B30000028E5D14EF604504FF08051CEF20000FF
:107B40000160BFF34F8FBFF36F8FD9E70498002810
:107B50009AD1BAF1000F18D04FF0500080F311887D
:107B6000BFF36F8FBFF34F8FFEE7BAF1000F0ED058
:107B7000FEF7DCFE606A20B1206B0068C0F13801BE
:107B800000E00021A068FFF7E5F9FEF7F5FE002010
:107B900005B0BDE8F08F000070B504460D466CB12D
:107BA000A66800F045F9864211D020462946FFF725
:107BB00011FF002804BF002070BD09E04FF0500005
:107BC00080F31188BFF36F8FBFF34F8FFEE7012063
:107BD000E1680131E16070BDB0B504460D46ACB15D
:107BE000EDB1FEF7A3FE40F2501CC2F2000CDCF82F
:107BF000142029684B1C1CD0D4E9000EDCF834306A
:107C0000834218D0724516D3012425E04FF050006E
:107C100080F31188BFF36F8FBFF34F8FFEE74FF0F4
:107C2000500080F31188BFF36F8FBFF34F8F00BFF9
:107C3000FEE7002410E0A2EB0E02914209D9881A57
:107C40002860DCF834002060DCF814006060002458
:107C500002E0002001242860FEF78EFE2046B0BD21
:107C60002DE9F04F81B09046824699460F464FEA83
:107C700088052846FEF7B8FB04465CB35C20FEF797
:107C8000B3FB06461EB3DDF828B000203463294656
:107C9000A52286F859002046F8F7E8FA306B002F45
:107CA00000EB8800A0F1040020F0070817D006F1CF
:107CB000340000217A5C42544A1C0F2A03D8795CB4
:107CC00000291146F6D1002086F843000AE020463C
:107CD000FEF76AFE4FF0FF3001B0BDE8F08F0020E4
:107CE00086F83400BBF1370F06F104004FF00004B2
:107CF00028BF4FF0370BC6F82CB0C6E913B4FEF717
:107D0000DDFD06F11800FEF7D9FDCBF13800366134
:107D100051464A46B06140467662746586F85840DE
:107D2000FEF740FC30600B98002818BF0660304614
:107D3000FDF7E0FF012001B0BDE8F08F2DE9F0472D
:107D400082B08246DDE90B04994615460F4640B3E2
:107D50008CB35C21019101995C2936D101990A9E6D
:107D60002063A522022184F85910A900F8F77EFAB1
:107D7000206B002F00EB8500A0F1040020F0070825
:107D80002DD004F1340000217A5C42544A1C0F2AA1
:107D900003D8795C00291146F6D1002084F843000D
:107DA00020E04FF0500080F31188BFF36F8FBFF3D6
:107DB0004F8F00BFFEE74FF0500080F31188BFF3F4
:107DC0006F8FBFF34F8F00BFFEE74FF0500080F37F
:107DD0001188BFF36F8FBFF34F8F00BFFEE7002006
:107DE00084F83400372E04F104004FF0000528BF5A
:107DF0003726E662C4E91365FEF760FD04F118005A
:107E0000FEF75CFDC6F13800246151464A46A06188
:107E100040466462656584F85850FEF7C3FB2060F5
:107E20002046FDF767FF204602B0BDE8F08700005E
:107E300040F6A840C2F200000068704740F25010BF
:107E4000C2F20000C168002904BF01207047016927
:107E50000020002908BF02207047000040F25010A7
:107E6000C2F200004069704780B5FEF70DFE40F297
:107E70005010C2F20000406980BD00002DE9F047BB
:107E800040F25016C2F20006306930B1306B002467
:107E9000013030632046BDE8F087706910F1010AB7
:107EA000C6F814A03ED0B06A824501D200244AE050
:107EB000B0690068002842D040F6AC4840F6A849B6
:107EC0000024C2F20008C2F2000900BFB069C06815
:107ED000C7683D4655F8040F824533D32846FEF760
:107EE000B3FCB86A00281CBF07F11800FEF7ACFC11
:107EF000F86A316A8842294688BF306200EB800008
:107F000008EB8000FEF7FCFCF86AD9F80010C96A9B
:107F1000884228BF0124B06900680028D6D14FF0FC
:107F2000FF300FE0B069006828B34FF0500080F3D5
:107F30001188BFF36F8FBFF34F8F00BFFEE74FF085
:107F4000FF300024B06240F6A84040F6AC41C2F2D7
:107F50000000C2F200010068C06A00EB800051F826
:107F60002000012888BF0124F06A002818BF0124DE
:107F70002046BDE8F087B069F169B161F061706BCE
:107F800001307063B069006820B1B069C068C06832
:107F9000406801E04FF0FF30B06284E72DE9F04324
:107FA00081B01E46154688460746FEF7BFFC40F6E0
:107FB000A844C2F20004206890F85800022845D076
:107FC0002068002E416D21EA070141654FF0010153
:107FD000206880F8581039D040F25019C2F20009D8
:107FE000D9F8147020680430FEF72EFC701C0FD0F6
:107FF00020683E44BE4246604FF0010028BF00208A
:1080000068B1D9F81C0021680431FEF75BFC12E06E
:10801000216809F14C000431FEF772FC0BE0D9F83D
:10802000180021680431FEF74DFCD9F8280086427B
:1080300038BFC9F828604EF604504FF08051CEF298
:1080400000000160BFF34F8FBFF36F8FFEF794FC0A
:10805000FEF76CFC002D1EBF2068406D28600025D7
:10806000206890F858100020022905D121680125C8
:108070004A6D22EA08024A65216881F85800FEF735
:108080007BFC284601B0BDE8F0830000B0B5044693
:10809000002C04BF0020B0BD40F6A840C2F2000092
:1080A0000068A04209D04FF0500080F31188BFF360
:1080B0006F8FBFF34F8F00BFFEE7206D38B30138DD
:1080C00020654FF0000018BFB0BDE16AE26C91423C
:1080D0001CD0251D2846FEF7B7FBE06CC0F1380127
:1080E000E062A16140F25011C2F200010A6A9042BE
:1080F00088BF086240F6AC4100EB8000C2F200018C
:1081000001EB80002946FEF7FBFB0120B0BD4FF0DC
:10811000500080F31188BFF36F8FBFF34F8F00BF04
:10812000FEE70000F0B581B00446002C02BF00203D
:1081300001B0F0BD40F6A846E06AC2F20006316820
:10814000C96A884216D2A16940F6AC4700EB8000AC
:10815000C2F2000707EB80000029A1BF3168C96A9D
:10816000C1F13801A161616981420CD03068C06AF7
:10817000E0621EE0E16C3068C26A0020914238BFC4
:10818000012001B0F0BD251D2846FEF75DFB3068DB
:1081900040F25011C2F20001C06AE0620A6A9042E5
:1081A00088BF086200EB8000294607EB8000FEF7DD
:1081B000A7FB012001B0F0BD70B5C068C5688DB1E6
:1081C00005F118042046FEF73FFB40F25016C2F2BC
:1081D0000006306978B106F160002146FEF790FB99
:1081E0002C351DE04FF0500080F31188BFF36F8FE6
:1081F000BFF34F8FFEE72C1D2046FEF725FB55F8F9
:108200002C0F316A884240F6AC4188BF306200EBE7
:108210008000C2F2000101EB80002146FEF770FBF6
:1082200040F6A8412868C2F200010968C96A88427C
:1082300092BF00200120F06270BD00002DE9F043E4
:1082400081B040F25015C2F20005286968B1FEF70E
:108250006DFB286901382861286980B10024FEF788
:108260008BFB204601B0BDE8F0834FF0500080F357
:108270001188BFF36F8FBFF34F8F00BFFEE7A86871
:10828000A0B3286EB8B340F6AC4940F6A8474FF00B
:108290000108C2F20009C2F2000700BFE86EC6681A
:1082A00006F11800FEF7D0FA341D2046FEF7CCFA8E
:1082B000F06A296A8842214688BF286200EB800064
:1082C00009EB8000FEF71CFBF06A3968C96A884236
:1082D00028BFC5F82C80286E0028DFD1A869006867
:1082E00030B1A869C068C068406803E00024B6E700
:1082F0004FF0FF30A8622C6B4CB10126FFF7BEFD9A
:10830000002818BFEE62013CF8D100202863E86A1B
:1083100060B14EF604504FF080510124CEF20000BF
:108320000160BFF34F8FBFF36F8F98E7002496E78C
:1083300070B586B0FEF7FAFA40F2D016C2F2000627
:10834000306810BB06F114042046FEF7ABFA06F1C4
:1083500028052846FEF7A6FA40F6084240F2705378
:1083600000201021C6E902450090C2F20002C2F2CC
:1083700000030A20FEF7C6FF0028306005D048F64B
:108380005031C0F60001FEF7B1FBFEF7F5FA306898
:10839000E0B1002004A903AACDE9040005A8FEF776
:1083A00073FADDE9032005990223CDE9003046F296
:1083B000311002910AA10023C0F60000FFF7BEFCB5
:1083C000002870601EBF012006B070BD4FF0500045
:1083D00080F31188BFF36F8FBFF34F8FFEE700BFAD
:1083E000546D7220537663004100080218BF0420C8
:1083F0000A0E18BF40F001004FF07F4232EA01013F
:1084000008BF40F00200012808BF0520704710EEA9
:10841000100A20F0004000EE100A704710EE101A0B
:1084200008B5444A6846B2EB410F28D94FF0E64000
:10843000B0EB410F94BF00204FF0FF300090009848
:10844000002861DB60EE000A10F0010F45D010F04B
:10845000020FDFED391A9FED391A00EEA11ADFED98
:10846000381A40EE811A21EEA01AF0EE400A40EED2
:10847000010A08BFF1EE600AB0EE600A08BD314B98
:1084800021F0004293423CD911F0004FDFED2E0A5B
:1084900020EE201ADFED2D0A19BF31EE601A71EEC1
:1084A000200A31EE201A71EE600ABDEEE01A11EEDC
:1084B000100A9FED271A00F0030000EEC10A9FED9D
:1084C000251A009000EEC10A9FED231A00EEC10AA2
:1084D0009FED221A00EEC10AB1E79FED211A9FED30
:1084E000210A10F0020F00EE810A9FED1F1A00EE24
:1084F000801AB7EE000A00EE810A18BFB1EE400AFA
:1085000008BD00F0F1F99AE710EE100A4000B0F152
:108510007F4F3CBFB7EE000A08BD07D14FF0010006
:1085200000F09CFABDE8084000F0CEB9BDE8084074
:1085300000F0C6B9B61F927E336D4CB9DA82083CA2
:10854000A0AA2ABE490E494683F9223F0000004BEB
:108550000000C93F00A0FD390020A2331A61342C6D
:10856000B93AB2BACA9F2A3DDDFFFFBE10B52DED64
:10857000028BB0EE608AF0EE408A18EE101A18EE08
:10858000900AF8F73FF800F07040B0F1005F0CD0AF
:1085900018EE100A20F00040C0F1FF40C00F02BFEB
:1085A000B0EE480ABDEC028B10BDB0EE680ABDEC1F
:1085B000028B10BD00B510EE101A2DED028B81B0AC
:1085C000524A6846B2EB410F2ED94FF0E640B0EB6D
:1085D000410F94BF00204FF0FF3000900098B0EEA4
:1085E000408A00286ADB10F0010F4BD068EE080AC1
:1085F0009FED471A9FED470A00EE810A9FED461A4C
:1086000010F0020F00EE801AB7EE000A00EE810AA9
:1086100002BF01B0BDEC028B00BD00BF01B0B1EEE6
:10862000400ABDEC028B00BD3C4B21F0004293425E
:1086300041D911F0004FDFED3A0A20EE201ADFEDAC
:10864000390A19BF31EE601A71EE200A31EE201A94
:1086500071EE600ABDEEE01A11EE100A9FED321ABB
:1086600000F0030000EEC10A9FED301A009000EE0A
:10867000C10A9FED2F1A00EEC10A9FED2E1A00EEDF
:10868000C10AABE728EE080A9FED2B1ADFED2B0A93
:1086900010F0020F40EE010A9FED291A00EE201A99
:1086A00061EE000AB0EE480A08EE200AB6D101B029
:1086B000BDEC028B00BD00F017F98FE718EE100A31
:1086C0004000B0F17F4F0DD218EE100AFFF78CFE7C
:1086D000042808BF00F000F9B0EE480A01B0BDEC74
:1086E000028B00BD09D1012000F0B8F901B0BDEC4A
:1086F000028B5DF804EB00F0E7B801B0B0EE480A79
:10870000BDEC028B5DF804EB00F0DAB8B61F927E88
:10871000B93AB2BACA9F2A3DDDFFFFBE490E4946AB
:1087200083F9223F0000004B0000C93F00A0FD3943
:108730000020A2331A61342C336D4CB9DA82083C24
:10874000A0AA2ABE00B510EE101A2DED028B81B042
:108750004D4A6846B2EB410F3CD94FF0E640B0EBD2
:10876000410F94BF00204FF0FF3000900098B0EE12
:10877000408A00285FDB28EE080ADFED440A9FEDFF
:10878000441A00EE201ADFED430A40EE010A9FED85
:10879000421A00EE201ADFED410A10F0010F40EE00
:1087A000010A9FED3F1A00EE201A61EE000AB0EEBA
:1087B000480A08EE200A02BF01B0BDEC028B00BDE2
:1087C000BFEE001A01B0C1EE000ABDEC028BB0EEA4
:1087D000600A00BD334B21F00042934228D911F0CA
:1087E000004FDFED310A20EE201ADFED300A19BF0D
:1087F00031EE601A71EE200A31EE201A71EE600A35
:10880000BDEEE01A11EE100A9FED291A00F00300E8
:1088100000EEC10A9FED271A009000EEC10A9FEDFD
:10882000261A00EEC10A9FED251A00EEC10A9DE747
:1088300000F05AF89AE718EE100A4000B0F17F4FA6
:108840000DD218EE100AFFF7CFFD042808BF00F084
:1088500043F8B0EE480A01B0BDEC028B00BD09D16F
:10886000012000F0FBF801B0BDEC028B5DF804EBD9
:1088700000F02AB801B0B0EE480ABDEC028B5DF8FA
:1088800004EB00F01DB80000B61F927EBCE9223C4C
:108890000B6D063B8A76CE3CACB5593D35A1083E02
:1088A00029AAAA3E490E494683F9223F0000004BFF
:1088B0000000C93F00A0FD390020A2331A61342C0A
:1088C00030EE000A70470000DFED020A80EEA00AD9
:1088D00070470000000000009FED020A20EE000A31
:1088E00070470000000000102DE9F0014FF07F42BA
:1088F000B2EB410F9FBF4FF0FF310160BDE8F001C7
:1089000070474FF0004242EA0123C1F3C752783A60
:10891000551112F01F0C434CCCF120067C44C1F3DE
:10892000C752A2F178024FEA621204EB820254F8B5
:10893000254008BFD2E9015612D0556804FA0CF45C
:1089400025FA06F73C43976805FA0CF527FA06F86E
:10895000D26807FA0CFCF24045EA08054CEA020628
:10896000A4FB034CA5FB0352A6FB03631D449D42DD
:1089700034BF012600261319334416B1934202D99D
:1089800003E0934201D2012200E00022624402F19E
:10899000200C9206DC0C42EA443200EE102A5B0303
:1089A000DFED210AF8EEC01A00EE103A4FEA9C1CE7
:1089B00011F0004FB8EE400AC0F800C020EE201AB7
:1089C00000EE105ADFED190AB8EE400A20EE200A38
:1089D00071EE810A70EE800A10EE902A02F50062B4
:1089E0006FF30B0200EE902A70EEE11A31EEC11A1D
:1089F000DFED101A30EE411A9FED0D0A20EE800ACD
:108A000001EE210A9FED0C1A00EE810A04BFBDE8B9
:108A1000F0017047CCF180510160BDE8F001B1EE8A
:108A2000400A704748010000000000360000802C1A
:108A300022AAFD29DB0FC92F0000C92F02E008C8B8
:108A4000121F08C1002AFAD170477047002001E0C8
:108A500001C1121F002AFBD17047000001490860C4
:108A60007047000004000020000000006E83F9A29F
:108A70002915444ED15727FCC0DD34F5999562DBAA
:108A80004190433CAB6351FE00401C4600008046D1
:108A90000060EA460000000000000000010203043C
:108AA0000607080900000000010203045F8B0008AC
:108AB00000000000000000000000000000000000B6
:108AC0000004000030000000000000000000000072
:108AD000698B00080000000000000000000000009A
:108AE000000000000004000018000000000000006A
:108AF00000000000558B000800000000000000008E
:108B00000000000000000000000400001800000049
:108B100000000000000000000006101600061016FD
:108B2000448B00080000000000000000000000006E
:108B3000000000000002000018000000000000001B
:108B40000000000064656661756C745461736B00AD
:108B5000546D72510079616F6B6F6E67716900546B
:108B600061736B5F496E6974007465737400000013
:108B7000908B000800000020900000003C8A000854
:108B8000208C000890000020C85F00004C8A00087C
:108B900000000000000000000100000010000000C4
:108BA000000000000024F4000000010201000000A9
:108BB00000000202010000000000030201000000AA
:108BC00000000402010000006F12833A000000411F
:108BD000CDCCCC3D0000003F0000FA4400007A46B6
:108BE0000000C842000080BF0000003F0000C040FD
:108BF00000000000CDCC4C3E0000803F0000004053
:108C00000000F041DB0FC9400000000000004842B6
:108C10000000484201000000AAAAAAAA0000000021
:040000050800018965
:00000001FF
